:020000040800F2
:1000000000060020F5050008B53400086D3400082E
:10001000953400086D3400088D340008F705000899
:10002000F7050008F7050008F705000899440008DF
:10003000F7050008F7050008F7050008F7050008B0
:10004000F7050008F7050008F7050008F7050008A0
:10005000F7050008F70500086974000895740008A2
:10006000C1740008ED74000819750008F705000850
:10007000F7050008F7050008F7050008F705000870
:10008000F7050008F7050008F70500084D340008DB
:10009000F70500085D340008F705000845750008FD
:1000A000F7050008F7050008F7050008F705000840
:1000B000F7050008F7050008F7050008F705000830
:1000C000F7050008F7050008F7050008F705000820
:1000D000F7050008F7050008F7050008F705000810
:1000E000A9750008F7050008F7050008F7050008DE
:1000F000F7050008F7050008F7050008F7050008F0
:10010000F7050008F705000831760008F705000834
:10011000F7050008F7050008F7050008F7050008CF
:10012000F7050008F7050008F7050008F7050008BF
:10013000F7050008F7050008F7050008F7050008AF
:10014000F7050008F7050008F7050008F70500089F
:10015000F7050008F7050008F7050008F70500088F
:10016000F7050008F7050008F7050008F70500087F
:10017000F70500081D6B0008F7050008F7050008E3
:10018000F7050008F70500081D760008F7050008C8
:10019000F7050008F7050008F7050008F70500084F
:1001A000F7050008F7050008F7050008F70500083F
:1001B000F7050008F7050008F7050008F70500082F
:1001C000F7050008F7050008F7050008F70500081F
:1001D000F7050008096B0008F7050008F705000897
:1001E000F7050008F7050008F7050008F7050008FF
:1001F000F7050008F7050008F7050008F7050008EF
:10020000F7050008F7050008F7050008F7050008DE
:10021000F7050008F7050008F7050008F7050008CE
:10022000F7050008F7050008F7050008F7050008BE
:10023000F7050008F7050008F7050008F7050008AE
:10024000F7050008F7050008F7050008F70500089E
:10025000F7050008F7050008F7050008F70500088E
:10026000F7050008F7050008F7050008F70500087E
:10027000F7050008F7050008F7050008F70500086E
:10028000F7050008F7050008F7050008F70500085E
:10029000F7050008F7050008F7050008F70500084E
:1002A000F7050008F7050008F7050008F70500083E
:1002B000F7050008F7050008F7050008F70500082E
:1002C000F7050008F7050008F7050008F70500081E
:1002D000F7050008F7050008F7050008F70500080E
:1002E000BD19000800000000000000000000000030
:1002F00053B94AB9002908BF00281CBF4FF0FF318D
:100300004FF0FF3000F074B9ADF1080C6DE904CE88
:1003100000F006F8DDF804E0DDE9022304B07047E0
:100320002DE9F047089D04468E46002B4DD18A42A8
:10033000944669D9B2FA82F252B101FA02F3C2F1DB
:10034000200120FA01F10CFA02FC41EA030E94406C
:100350004FEA1C48210CBEFBF8F61FFA8CF708FB8D
:1003600016E341EA034306FB07F199420AD91CEB65
:10037000030306F1FF3080F01F81994240F21C8197
:10038000023E63445B1AA4B2B3FBF8F008FB1033DF
:1003900044EA034400FB07F7A7420AD91CEB040414
:1003A00000F1FF3380F00A81A74240F207816444E4
:1003B000023840EA0640E41B00261DB1D440002369
:1003C000C5E900433146BDE8F0878B4209D9002DCD
:1003D00000F0EF800026C5E9000130463146BDE857
:1003E000F087B3FA83F6002E4AD18B4202D38242C1
:1003F00000F2F980841A61EB030301209E46002D70
:10040000E0D0C5E9004EDDE702B9FFDEB2FA82F2C4
:10041000002A40F09280A1EB0C014FEA1C471FFA22
:100420008CFE0126200CB1FBF7F307FB131140EA09
:1004300001410EFB03F0884208D91CEB010103F1D6
:10044000FF3802D2884200F2CB804346091AA4B298
:10045000B1FBF7F007FB101144EA01440EFB00FE6C
:10046000A64508D91CEB040400F1FF3102D2A645D1
:1004700000F2BB800846A4EB0E0440EA03409CE770
:10048000C6F12007B34022FA07FC4CEA030C20FA1D
:1004900007F401FA06F31C43F9404FEA1C4900FA3D
:1004A00006F3B1FBF9F8200C1FFA8CFE09FB1811BA
:1004B00040EA014108FB0EF0884202FA06F20BD92D
:1004C0001CEB010108F1FF3A80F08880884240F27D
:1004D0008580A8F102086144091AA4B2B1FBF9F0C1
:1004E00009FB101144EA014100FB0EFE8E4508D9BC
:1004F0001CEB010100F1FF346CD28E456AD9023841
:10050000614440EA0840A0FB0294A1EB0E01A14225
:10051000C846A64656D353D05DB1B3EB080261EB93
:100520000E0101FA07F722FA06F3F1401F43C5E96D
:10053000007100263146BDE8F087C2F12003D840A3
:100540000CFA02FC21FA03F3914001434FEA1C47E5
:100550001FFA8CFEB3FBF7F007FB10360B0C43EAD7
:10056000064300FB0EF69E4204FA02F408D91CEB87
:10057000030300F1FF382FD29E422DD90238634485
:100580009B1B89B2B3FBF7F607FB163341EA034125
:1005900006FB0EF38B4208D91CEB010106F1FF3874
:1005A00016D28B4214D9023E6144C91A46EA00466B
:1005B00038E72E46284605E70646E3E61846F8E6FD
:1005C0004B45A9D2B9EB020864EB0C0E0138A3E746
:1005D0004646EAE7204694E74046D1E7D0467BE727
:1005E000023B614432E7304609E76444023842E79F
:1005F000704700BF02E000F000F8FEE772B637482F
:1006000080F30888364880F3098836483649086000
:1006100040F20000CCF200004EF63471CEF2000140
:100620000860BFF34F8FBFF36F8F40F20000C0F23E
:10063000F0004EF68851CEF200010860BFF34F8FF4
:10064000BFF36F8F4FF00000E1EE100A4EF63C71E1
:10065000CEF200010860062080F31488BFF36F8F8C
:1006600005F0D2FC06F0D6FC4FF055301F491B4A6E
:1006700091423CBF41F8040BFAE71D49184A9142E8
:100680003CBF41F8040BFAE71A491B4A1B4B9A423C
:100690003EBF51F8040B42F8040BF8E7002018495C
:1006A000184A91423CBF41F8040BFAE705F0EAFC16
:1006B00006F032FD144C154DAC4203DA54F8041B1D
:1006C0008847F9E700F042F8114C124DAC4203DACA
:1006D00054F8041B8847F9E705F0D2BC0006002057
:1006E000002200200000000808ED00E000000020CB
:1006F00000060020D07B000800220020D02200202D
:10070000D022002080720020E0020008E4020008ED
:10071000E4020008E40200082DE9F04F2DED108AF4
:10072000C1F80CD0D0F80CD0BDEC108ABDE8F08F29
:10073000002383F311882846A047002004F04EFFD1
:10074000FEE704F0A7FE00DFFEE70000F8B501F0C9
:1007500047F905F0DDFB074605F04CFC0546B8BB44
:10076000204B9F4234D001339F4234D027F0FF0208
:100770001D4B9A4232D12E4642F21074F8B200F06C
:100780006DFF00F071FF08B10024264601F02AFD3C
:1007900020B10024032000F07BF8264635B1134B2E
:1007A0009F4203D0002405F01DFC2646002005F0E2
:1007B000B9FB0EB100F082F801F0C0FA00F088FF3A
:1007C00001F08AF9204600F01DF900F077F8F9E70A
:1007D0002E460024D5E704460126D2E7064641F21C
:1007E0008834CEE7010007B0000008B0263A09B00F
:1007F00008B501F03DF9A0F120035842584108BD69
:1008000007B541F21203022101A8ADF8043001F04E
:100810004DF903B05DF804FB38B5302383F311883C
:10082000174803680BB104F0A5FF0023154A4FF4E5
:100830007A71134804F094FF002383F31188124C5B
:10084000236813B12368013B2360636813B16368B5
:10085000013B63600D4D2B7833B963687BB902208F
:1008600001F0EEF9322363602B78032B07D1636824
:100870002BB9022001F0E4F94FF47A73636038BDBC
:10088000D022002019080008F0230020E8220020D0
:10089000084B187003280CD8DFE800F008050208A0
:1008A000022001F0CBB9022001F0C6B9024B0022B0
:1008B0005A607047E8220020F0230020F8B501F0CC
:1008C00091FC30B1464B03221A700022454B5A600E
:1008D000F8BD454B454A1C4619680131F8D0043330
:1008E0009342F9D16268424B9A42F1D9414B9B68DD
:1008F00003F1006303F580239A42E9D205F046FB39
:1009000005F058FB002001F00DF90220FFF7C0FFB1
:10091000394B00219A6C99641A6F19671A6FDA6C57
:10092000D9645A6F59675A6F1A6D19659A6F99672A
:100930009B6F324BD3F8802042F00072C3F88020C6
:10094000D3F8802022F00072C3F88020D3F88030E2
:1009500072B64FF0E023C3F8084DD4E90004BFF3AA
:100960004F8FBFF36F8F264AC2F88410BFF34F8FAB
:10097000536923F480335361BFF34F8FD2F8803033
:1009800043F6E076C3F3C905C3F34E335B0103EAD4
:10099000060C29464CEA81770139C2F87472F9D203
:1009A000203B13F1200FF2D1BFF34F8FBFF36F8FB6
:1009B000BFF34F8FBFF36F8F536923F4003353613D
:1009C0000023C2F85032BFF34F8FBFF36F8F302335
:1009D00083F31188854680F30888204778E700BFB5
:1009E000E8220020F0230020000004082000040872
:1009F000FFFF03080022002000450258004402586F
:100A000000ED00E02DE9F04F93B0B74B2022FF211D
:100A100000900AA89D6801F03BF9B44A1378A3B985
:100A20000121B34811700360302383F311880368F8
:100A30000BB104F09FFE0023AE4A4FF47A71AC482C
:100A400004F08EFE002383F31188009B13B1AA4BA0
:100A5000009A1A60A94A1378032B03D0002313705D
:100A6000A54A53604FF0000A009CD3465646D14633
:100A7000012001F0E3F824B19F4B1B68002B00F02C
:100A80002C82002000F0F4FF0390039B002B01DA7E
:100A900000F066FE039B002BEDDB012001F0CCF89B
:100AA000039B213B1F2BE3D801A252F823F000BF88
:100AB000310B0008590B0008ED0B0008710A000803
:100AC000710A0008710A00087F0C00084F0E000828
:100AD000690D0008CB0D0008F30D0008190E000881
:100AE000710A00082B0E0008710A00089D0E00080C
:100AF000D10B0008710A0008E10E00083D0B000848
:100B0000D10B0008710A0008CB0D0008710A00081B
:100B1000710A0008710A0008710A0008710A0008C9
:100B2000710A0008710A0008710A0008ED0B00083C
:100B30000220FFF75DFE002840F0F981009B0221B2
:100B400005A8BAF1000F08BF1C4641F21233ADF8F8
:100B5000143000F0ABFF8BE74FF47A7000F088FFA1
:100B6000071EEBDB0220FFF743FE0028E6D0013F23
:100B7000052F00F2DE81DFE807F0030A0D101336BF
:100B80000523042105A8059300F090FF17E0042138
:100B90005548F9E704215A48F6E704215948F3E794
:100BA0004FF01C08404608F1040800F0BDFF042186
:100BB000059005A800F07AFFB8F12C0FF2D10120C2
:100BC0004FF0000900FA07F747EA0B0B5FFA8BFBBF
:100BD00001F0AAF826B10BF00B030B2B08BF002481
:100BE000FFF70EFE44E704214748CDE7002EA5D0CD
:100BF0000BF00B030B2BA1D10220FFF7F9FD0746E9
:100C000000289BD00120002600F08CFF0220FFF777
:100C10003FFE1FFA86F8404600F094FF0446B0B14C
:100C2000039940460136A1F140025142514100F082
:100C3000A1FF0028EDD1BA46044641F21213022169
:100C400005A83E46ADF8143000F030FF10E7254609
:100C50000120FFF71DFE244B9B68AB4207D92846B5
:100C600000F062FF013040F067810435F3E70025B2
:100C7000224BBA463E461D701F4B5D60A8E7002E12
:100C80003FF45CAF0BF00B030B2B7FF457AF02204C
:100C9000FFF7FEFD322000F0EBFEB0F10008FFF69A
:100CA0004DAF18F003077FF449AF0F4A08EB050377
:100CB000926893423FF642AFB8F5807F3FF73EAF70
:100CC000124BB845019323DD4FF47A7000F0D0FE4B
:100CD0000390039A002AFFF631AF039A0137019B74
:100CE00003F8012BEDE700BF00220020EC230020D9
:100CF000D022002019080008F0230020E82200205C
:100D000004220020082200200C220020EC220020D7
:100D1000C820FFF76DFD074600283FF40FAF1F2DD9
:100D200011D8C5F120020AAB25F0030084494245E1
:100D3000184428BF4246019200F084FF019AFF2127
:100D40007F4800F0A5FF4FEAA803C8F387027C495B
:100D50002846019300F0A4FF064600283FF46DAF3B
:100D6000019B05EB830533E70220FFF741FD0028D7
:100D70003FF4E4AE00F010FF00283FF4DFAE0027A0
:100D8000B846704B9B68BB4218D91F2F11D80A9BDD
:100D900001330ED027F0030312AA134453F8203C6A
:100DA00005934046042205A9043701F005FA804660
:100DB000E7E7384600F0B8FE0590F2E7CDF814807A
:100DC000042105A800F072FE02E70023642104A8B4
:100DD000049300F061FE00287FF4B0AE0220FFF71C
:100DE00007FD00283FF4AAAE049800F0CBFE059062
:100DF000E6E70023642104A8049300F04DFE0028D8
:100E00007FF49CAE0220FFF7F3FC00283FF496AE7F
:100E1000049800F0B9FEEAE70220FFF7E9FC002899
:100E20003FF48CAE00F0C8FEE1E70220FFF7E0FCE3
:100E300000283FF483AE05A9142000F0C3FE074646
:100E40000421049004A800F031FE3946B9E73220AD
:100E500000F00EFE071EFFF671AEBB077FF46EAE0C
:100E6000384A07EB0903926893423FF667AE0220C7
:100E7000FFF7BEFC00283FF461AE27F003074F44A4
:100E8000B9453FF4A5AE484609F1040900F04CFE0F
:100E90000421059005A800F009FEF1E74FF47A70EF
:100EA000FFF7A6FC00283FF449AE00F075FE0028CD
:100EB00044D00A9B01330BD008220AA9002000F07D
:100EC000EFFE00283AD02022FF210AA800F0E0FE21
:100ED000FFF796FC1C4804F087FB13B0BDE8F08FC9
:100EE000002E3FF42BAE0BF00B030B2B7FF426AE42
:100EF0000023642105A8059300F0CEFD07460028D5
:100F00007FF41CAE0220FFF773FC804600283FF4FC
:100F100015AEFFF775FC41F2883004F065FB0598CB
:100F200000F04CFF46463C4600F0FEFEA0E50646BB
:100F30004EE64FF0000901E6BA467EE637467CE60B
:100F4000EC22002000220020A0860100094A49F27C
:100F50006900136899B21B0C00FB013344F2506125
:100F60001360054B186882B2000C01FB0200186088
:100F700080B270471422002010220020002110228D
:100F800010B5044600F084FE034B03CB2060616083
:100F90001868A06010BD00BF00E8F11F2DE9F04106
:100FA000ADF5507D0D46002140F275126EAC07463E
:100FB00010A80F9100F06CFE4FF4C472002120467F
:100FC00000F066FE0DF13C0802F07CFA4FF47A72F4
:100FD000264BB0FBF2F0186093E80700022384E888
:100FE00007000DF5ED702382FFF7C8FF43F204738D
:100FF0001F4907A8238406F0BFFB1E230DF2EB2236
:101000000DF1340C84F8323107AB1E46083203CEA2
:10101000664542F8080C42F8041C3346F5D13068A6
:10102000414610602046B3889380012200F0E8FE1C
:10103000002380B2E97E0393AB7E029305F119038E
:1010400001930123009307A3D3E90023CDE9048092
:10105000384602F0F5FD0DF5507DBDE8F08100BF8A
:10106000AFF300809E6AC421818A46EEF8230020F7
:10107000887700082DE9F0412C4CDAB080460D4607
:10108000237A5BBB27A9284600F0C8FF0746002843
:1010900042D19DF89D60C82E3ED801464FF4A6620D
:1010A000204600F0F5FD4FF4807332460DF19E01AD
:1010B000C4F8F8314FF4007304F109002644C4F871
:1010C0000C334FF44073C4F8203400F0BBFD9DF89E
:1010D0009C30777223720BB9EB7E237206AC8122AF
:1010E000002127A800F0D4FD0122214627A800F006
:1010F000D1FF002380B2E97E0393AB7E029305F11A
:10110000190301932823CDE904400093404605A329
:10111000D3E9002302F094FD5AB0BDE8F08100BF8E
:10112000AFF3008026417272DF25D7B7F048002068
:10113000F0B5254E4FF48A75F1B0002405FB00652B
:1011400096F8D830D822214685F8DC303AA885F8C0
:10115000E84006AF00F09CFD06F1090000F090FDAC
:10116000D5F8E430C2B206F109018DF8F0000DF1B6
:10117000F100CDE93A3400F065FD394601223AA884
:1011800000F0B4FF082380B2317ACDE90470012762
:101190000E48CDE9023706F1D803019330230093BE
:1011A00007A3D3E9002302F04BFDA04206DD02F0C5
:1011B00089F9C5F8E000384671B0F0BD2046FBE77C
:1011C00078F6339F93CACD8DF0480020103400206C
:1011D0002DE9F0411D4D86B01D4E1E4F284602F0F0
:1011E0005BFD034658B30024DFF86C80ADF8144073
:1011F0000294CDE90344027B8DF8142003AA996878
:10120000406803C21B6843F00043029302F05CF99C
:1012100082190094384641F1000302A901F0E4F973
:10122000A04205DD284602F03BFD88F80040D5E7E6
:1012300098F80030072B05D8013388F8003006B045
:10124000BDE8F081014802F02BFDF8E710340020E2
:1012500040420F0040340020254E002070B50D465E
:1012600014461E4602F048FC50B9022E10D1012C43
:101270000ED112A3D3E900230120C5E9002307E022
:10128000282C10D005D8012C09D0052C0FD0002017
:1012900070BD302CFBD10BA3D3E90023ECE70BA3EB
:1012A000D3E90023E8E70BA3D3E90023E4E70BA38A
:1012B000D3E90023E0E700BFAFF30080401DA12089
:1012C00026812A0B78F6339F93CACD8D9E6AC4215E
:1012D000818A46EE26417272DF25D7B7F017304A71
:1012E00039059E5638B505460E4C0021013500F0F3
:1012F00041FCA4F82C55B4F82C0500F023FC78B17F
:10130000B4F82C0500F02EFC014648B9B4F82C05C1
:1013100000F030FCB4F82C350133A4F82C35EAE7A2
:1013200038BD00BFF04800200A4B0B4A10B51A60C8
:1013300003F5805393F848203AB95C6C2CB12046F1
:1013400000F0CEFF204606F0CDF90448BDE810407D
:1013500000F0C6BF403400203878000870440020F8
:101360002DE9F04F8FB005460C4600AF02F0C4FBEC
:10137000002849D1237E022B1BD1E38A012B18D1EF
:1013800002F0A0F80646FFF7E1FD03464FF4C870EF
:1013900006F51676DFF8C082B3FBF0F202FB1033DD
:1013A00016FA83F3C8F80030E37E33B9A34B00226A
:1013B0001A703C37BD46BDE8F08F07F12401204686
:1013C00000F0EAFD0028F4D107F11400FFF7D6FD84
:1013D00097F8264007F1140107F12700224606F08E
:1013E00099F90028E2D10F2C08D8944B1C70D8F83A
:1013F0000030A3F51673C8F80030DAE797F8241028
:10140000284602F071FBD4E7E38A282B2BD010D8B2
:10141000012B23D0052BCCD1BFF34F8F8849894BAB
:10142000CA6802F4E0621343CB60BFF34F8F00BF82
:10143000FDE7302BBDD1844EE17E327A9142B8D1A6
:10144000607E3146002291F8DC50854200F0A58094
:10145000013201F58A71042AF5D1AAE7214628460E
:10146000FFF79CFDA5E721462846FFF703FEA0E70E
:10147000B2F8EC507B6005F103094FEA99094FEA95
:101480008902D11DC908A8EBC10300219D46EB4686
:10149000584600F0FDFB04F1EE012A46584631445F
:1014A00000F0D0FB7B6813B9012000F03BFB96F8FD
:1014B000D20000F047FB044630B9307200F06CFBFC
:1014C000204600F02FFBB1E0D6F8D4203AB996F8C8
:1014D000D200B6F82C25824201D8FFF703FFD6F8D8
:1014E000D4202A44944208D296F8D200B6F82C258B
:1014F0000130824201D8FFF7F5FE5FFA89F25946C2
:10150000706800F0CDFB08B9C54679E0726896F8BE
:10151000D2002A447260D6F8D42005EB0209C6F83E
:10152000D49000F00FFB814509D396F8D220D6F86D
:10153000D4000132001B86F8D220C6F8D400FF2D5B
:101540000FD80024347200F027FB204600F0EAFA9E
:1015500000F048FE3D4B188108B9FFF7AFF9C546CA
:1015600027E7BB6896F8D9000AFB0362FB68D2F84C
:10157000E41082F8E83001F58061C2F8E030C2F88A
:10158000E410FFF7D5FDFFF723FE96F8D9200132CE
:1015900002F0030286F8D920B6E74FF48A7A204693
:1015A0000AFB02F505F1EA01314400F0CBFDF860D9
:1015B00000287FF4FEAE0122354485F8E82001F0D2
:1015C00081FFD5F8E020D6ED007A801A40F6B832D7
:1015D000B8EE677ADFED1E6A192838BF19209042ED
:1015E00028BF104607EE900AF8EEE77A67EEA67A73
:1015F000DFED186AE7EE267AFCEEE77AC6ED007AB0
:1016000096F8D930BB60BA6873680AFB02F43219E5
:1016100092F8E81059B1D2F8E410E8468B423FF452
:1016200027AF002182F8E810C2F8E010C5467368C1
:10163000064A9B0A01331381BBE600BF0934002030
:1016400000ED00E00400FA05F0480020F823002037
:10165000CDCCCC3D6666663F0C340020014B187043
:10166000704700BF0424002038B54FF04054144B9D
:1016700022689A4221D1627D0025124B12481A70CD
:10168000C922237D0930114900F8013C4FF48073D1
:10169000C0F8DB50C0F8EF314FF40073C0F80333EB
:1016A0004FF44073C0F8173400F0CCFAE02229461A
:1016B000204600F0EDFA012038BD0020FCE700BF15
:1016C0009AAD44C504240020F048002016000030E4
:1016D00037B500F087FD194D0223002218492881F3
:1016E0006B710123174801F0D9FA002316494FF412
:1016F00080520193154B16480093164B02F0CCF91B
:10170000154B197811B1124802F0EEF901F0DAFE2A
:101710000446FFF71BFC4FF4C873B0FBF3F202FB67
:10172000130304F5167010FA83F00C4B186004F0E4
:1017300061FC08B10F232B8103B030BDF8230020DA
:1017400040420F0040340020082400205D120008B1
:101750001034002061130008042400200C34002001
:101760002DE9F04F8C4C2DED028B85A7D7E9006752
:1017700095B00FF21429D9E900899FED858BFFF709
:1017800027FD0DAD0023DFF824B20C93ADF83C30FB
:101790000D936B6000234FF0010A0DF1250209A99A
:1017A00058468DF825308DF824A08DED008B01F082
:1017B000F1FD9DF824200023002A40F0AE80204651
:1017C00002F09AF90546002847D1DFF8E4B101F0AC
:1017D00079FEDBF8003098423FD301F073FE0790AA
:1017E000FFF7B4FB4FF4C873079AB0FBF3F101FBAA
:1017F000130302F5167010FA83F0CBF8000010A85E
:10180000DFF8B0B19BF80010002914BF2B465346F7
:1018100007918DF83030FFF7B1FB079910AB0DF150
:101820003100C1F110021944D2B2062A28BF0622A3
:10183000079200F007FA079A0CAB20460393013297
:101840001823D2B20293554B04923246CDE900A33D
:101850003B4602F097F98BF8005001F033FE504AF6
:10186000504D1368C31AB3F57A7F32D3106001F07C
:101870002BFE02460B46204602F01CFA204602F0E0
:101880003BF930B32B7A0DF1400BDFF82CA1002B84
:1018900014BF032302238AF8053001F013FE4FF42E
:1018A0007A7301225946B0FBF3F0CAF800005046A3
:1018B00000F04AFB182380B2424602933A4B019350
:1018C00040F25513CDE903B0009320464B4602F099
:1018D00059F92B7AABB101F0F5FD4FF0000A8346C0
:1018E0004FF48A7295F8D900504400F0030002FBCF
:1018F000005393F8E81071B30AF1010ABAF1040F2A
:10190000F0D1C82003F070FE2B7A002B7FF435AFA6
:1019100015B0BDEC028BBDE8F08F1946102210A85F
:1019200000F0B6F90DF126030AAA0CA9584601F0F9
:1019300063F811AB95E8030083E803009DF83C30A1
:1019400010A920468DF84C300C9B1093DDE90A233A
:1019500002F084FB1EE7D3F8E01049B12B68ABEB33
:101960000101FA2B38BFFA230533B1EB430FC3D380
:10197000FFF7DEFB4FF48A720028BDD1C1E700BF3C
:10198000401DA12026812A0BF1C6A7C1D068080FEF
:101990000000000000000000103400200834002087
:1019A000204E0020F0480020244E0020403400202B
:1019B0000C34002009340020F823002008B5054825
:1019C00001F0C0F8044A05490020BDE8084005F0D0
:1019D00083BE00BF403400207C4E00202913000845
:1019E000704700002DE9F84F4FF47A7306460D4614
:1019F000002402FB03F7DFF85080DFF8509098F9DD
:101A000000305FFA84FA5A1C01D0A34212D159F86F
:101A100024002A4631460368D3F820B03B46D84715
:101A2000854207D1074B012083F800A0BDE8F88F5D
:101A30000124E4E7002CFBD04FF4FA7003F0D4FD4E
:101A40000020F3E76C4E0020182200201C2200200A
:101A500070B504464FF47A76412C254628BF4125BF
:101A600006FB05F003F0C0FD641BF5D170BD00005E
:101A7000002307B5024601210DF107008DF807305C
:101A8000FFF7B0FF20B19DF8070003B05DF804FB3D
:101A90004FF0FF30F9E700000A46042108B5FFF7D0
:101AA000A1FF80F00100C0B2404208BD074B0A46CA
:101AB00030B41978064B53F821400146236820467C
:101AC000DD69044BAC4630BC604700BF6C4E002063
:101AD0001C220020A086010070B5104C0025104E7D
:101AE00004F09CF820803068238883420CD80025BD
:101AF0002088013804F08EF823880544013BB5F5B1
:101B0000802F2380F4D370BD04F084F8336805443B
:101B10000133B5F5802F3360E5D3E8E76E4E002042
:101B2000284E002004F048B900F1006000F5802044
:101B30000068704700F10060920000F5802004F01A
:101B4000C9B80000054B1A68054B1B889B1A8342D5
:101B500002D9104404F05EB800207047284E0020DF
:101B60006E4E0020024B1B68184404F059B800BFA9
:101B7000284E0020024B1B68184404F063B800BFD5
:101B8000284E00200020704700F1FF5000F58F1014
:101B9000D0F8000870470000064991F8243033B1AE
:101BA00000230822086A81F82430FFF7C3BF012010
:101BB000704700BF2C4E0020014B1868704700BFD3
:101BC0000010005C194B01380322084470B51D68F1
:101BD000174BC5F30B042D0C1E88A6420BD15C6875
:101BE0000A46013C824213460FD214F9016F4EB1EE
:101BF00002F8016BF6E7013A03F10803ECD18142E8
:101C00000B4602D22C2203F8012B0424094A168821
:101C1000AE4204D1984284BF967803F8016B013C30
:101C200002F10402F3D1581A70BD00BF0010005C2D
:101C300024220020D477000870470000704700007D
:101C400070470000002310B5934203D0CC5CC4540D
:101C50000133F9E710BD0000013810B510F9013F5C
:101C60003BB191F900409C4203D11AB10131013AD4
:101C7000F4E71AB191F90020981A10BD1046FCE75C
:101C800003460246D01A12F9011B0029FAD1704707
:101C900002440346934202D003F8011BFAE770475F
:101CA0002DE9F8431F4D14460746884695F8242031
:101CB00052BBDFF870909CB395F824302BB92022EA
:101CC000FF2148462F62FFF7E3FF95F824004146C5
:101CD000C0F1080205EB8000A24228BF2246D6B21E
:101CE0009200FFF7AFFF95F82430A41B17441E4461
:101CF0009044E4B2F6B2082E85F82460DBD1FFF7F9
:101D00004BFF0028D7D108E02B6A03EB8203834204
:101D1000CFD0FFF741FF0028CBD10020BDE8F883EA
:101D20000120FBE72C4E0020024B1A78024B1A7060
:101D3000704700BF6C4E00201822002038B51A4CA6
:101D40001A4D204602F06EFF2946204602F096FF0B
:101D50002D684FF47A70D5F89020D2F8043843F00B
:101D60000203C2F80438FFF773FE1149284603F056
:101D700093F8D5F890200F4DD2F80438286823F056
:101D800002030D49A042C2F804384FF4E1330B605E
:101D900001D002F0A5FE6868A04204D00649BDE863
:101DA000384002F09DBE38BD6055002064790008BF
:101DB0006C7900081C220020544E00200C4B70B59A
:101DC0000C4D04461E780C4B55F826209A420DD037
:101DD0000A4B002118221846FFF75AFF04600146FB
:101DE00055F82600BDE8704002F07ABE70BD00BF15
:101DF0006C4E00201C22002060550020544E002014
:101E00002DE9F0470D46044600219046284640F251
:101E10007912FFF73DFF234620220021284604F1D6
:101E2000220702F0BDF8231D022220212846C026E9
:101E300002F0B6F8631D03222221284602F0B0F812
:101E4000A31D03222521284602F0AAF804F1080365
:101E500010222821284602F0A3F804F110030822DA
:101E60003821284602F09CF804F111030822402191
:101E7000284602F095F804F112030822482128466A
:101E800002F08EF804F1140320225021284602F0BB
:101E900087F804F1180340227021284602F080F8E8
:101EA00004F120030822B021284602F079F804F159
:101EB00021030822B821284602F072F8314608367C
:101EC0003B4608222846013702F06AF8B6F5A07FA3
:101ED000F4D1002704F1330A04F132030822314619
:101EE000284602F05DF894F832304FEAC7099F4265
:101EF00009F5A47615D3B8F1000F08D1314609F2DF
:101F00004F1604F599730722284602F049F8274630
:101F10003B1B94F8322193420CD3F01DC008BDE85E
:101F2000F0870AEB0703082231462846013702F002
:101F300037F8D8E707F23313314608222846083627
:101F4000013702F02DF8E3E713B5044608460021F7
:101F50002022234601900160C0F8031002F020F80F
:101F6000231D01980222202102F01AF8631D019816
:101F70000322222102F014F8A31D01980322252137
:101F800002F00EF8019804F108031022282102F053
:101F900007F8072002B010BD0023F7B50E46047FF6
:101FA000072200911946054601F0BEFE731C01226E
:101FB000072100932846002301F0B6FEC4B9B31CE4
:101FC000052208212846009323460D2401F0ACFE8B
:101FD0003746BB1BB278934211D307342B7FA88AB4
:101FE000E408BBB9844294BF0020012003B0F0BDD7
:101FF000AB8A0824DB00083BDB08B370E8E7FB1C76
:10200000214608222846009300230834013701F0B6
:102010008BFEDEE7201A18BF0120E7E70023F7B5A3
:102020000E46047F082200911946054601F07CFE09
:10203000731CC4B908220093234610241146284675
:1020400001F072FE01235F1C7278013B934211D3B1
:1020500007342B7FA88AE408BBB9844294BF0020D0
:10206000012003B0F0BDAB8A0824DB00083BDB088D
:102070007370E7E7F31921460822284600930023EE
:1020800001F052FE08343B46DDE7201A18BF01205C
:10209000E7E70000F8B50E46054614460021812208
:1020A0003046FFF7F5FD2B4608220021304601F0AF
:1020B00077FF7CB90F246B1C07220821304601F002
:1020C0006FFF01235F1C6A78013B934204D3E01D3C
:1020D000C008F8BD0824F4E7EB1921460822304671
:1020E00001F05EFF08343B46ECE70000F8B50E4611
:1020F000054614460021CE223046FFF7C9FD2B4687
:1021000028220021304601F04BFF7CB9302405F134
:10211000080308222821304601F042FF2F467B1B8E
:102120002A7A934204D3E01DC008F8BD2824F5E7BD
:1021300007F109032146082230460834013701F02F
:102140002FFFECE7F7B5047F0E4600910123102224
:102150000021054601F0E8FDC4B9B31C0922102195
:10216000284600932346192401F0DEFD3746728885
:10217000BB1B9A4211D807342B7FA88AE408BBB94D
:10218000844294BF0020012003B0F0BDAB8A10242C
:10219000DB00103BDB087380E8E73B1D214608228B
:1021A0002846009300230834013701F0BDFDDEE727
:1021B000201A18BF0120E7E730B50A44084D9142C4
:1021C0000DD011F8013B5840082340F30004013BB7
:1021D0002C4013F0FF0384EA5000F6D1EFE730BD46
:1021E0002083B8EDF7B5384A6B46106851686A46E7
:1021F00003C308233549364805F09CFA04460028F5
:1022000033D10A25334A6B46106851686A4603C3C6
:10221000082331492E4805F08DFA0446002849D09C
:102220000369B3F5E01F45D8B0F8661040F23742B5
:1022300091423FD1294A024402F15C018B4239D3D9
:102240005C3B234900209E1AFFF7B6FF04F16401AE
:10225000074632460020FFF7AFFFA3689F4229D10F
:10226000E368984208BF002524E00369B3F5E01F46
:1022700027D8418B40F23742914220D1174A02447D
:1022800002F110018B4218D3103B114900209D1A16
:10229000FFF792FF04F1180106462A460020FFF7D7
:1022A0008BFFA3689E4202D1E368984201D00D25BE
:1022B000A8E70025284603B0F0BD1025A2E70C25AD
:1022C000A0E70B259EE700BFE4770008DCFF1B00BA
:1022D00000000408ED77000890FF1B000800FCF7E1
:1022E00010B5037C044613B9006805F00BFA2046CC
:1022F00010BD00000023BFF35B8FC360BFF35B8F93
:10230000BFF35B8F8360BFF35B8F7047BFF35B8F5F
:102310000068BFF35B8F704770B505460C30FFF760
:10232000F5FF044605F108063046FFF7EFFFA0422F
:1023300006D96D683046FFF7E9FF2544281A70BDBD
:102340003046FFF7E3FF201AF9E7000070B50546B5
:102350004068A0B105F10C0605F10800FFF7D6FFB3
:1023600004463046FFF7D2FF844204F1FF34304682
:1023700094BF6D680025FFF7C9FF2C44201A70BD7B
:1023800038B50C460546FFF7C7FFA04210D305F14C
:102390000800FFF7BBFF04446868BFF35B8FB4FB22
:1023A000F0F100FB11440120AC60BFF35B8F38BD3E
:1023B0000020FCE72DE9F041144607460D46FFF7E3
:1023C000C5FF844228BF0446D4B1B84658F80C6B08
:1023D0004046FFF79BFF3044286040467E68FFF789
:1023E00095FF331A9C4203D801206C60BDE8F08150
:1023F000A41B6B603B682044AB60E8600220F5E7FB
:102400002046F3E738B50C460546FFF79FFFA0428C
:1024100010D305F10C00FFF779FF04446868BFF39F
:102420005B8FB4FBF0F100FB11440120EC60BFF3C3
:102430005B8F38BD0020FCE72DE9FF4188466946E7
:1024400007466C46FFF7B6FF002506B204EBC6064A
:10245000B4420AD0626808EB050120680834FFF72F
:10246000F1FB54F8043C1D44F2E729463846FFF7D7
:10247000C9FF284604B0BDE8F0810000F8B5054664
:102480000C300F46FFF742FF05F1080604463046C0
:10249000FFF73CFFA042304688BF6C68FFF736FF6D
:1024A000201A386020B12C683046FFF72FFF2044F7
:1024B000F8BD000073B5144606460D46FFF72CFF25
:1024C0008442019028BF0446DCB101A93046FFF7E1
:1024D000D5FF019B33B93268C5E90233C5E9002451
:1024E00001200CE09C42286038BF0194019884428E
:1024F0006860F5D93368241A0220AB60EC6002B042
:1025000070BD2046FBE700002DE9FF410F466946FC
:102510006C46FFF7CFFF00B2002604EBC005AC42CB
:1025200009D0D4F80480B81954F8081B4246464430
:10253000FFF788FBF3E7304604B0BDE8F081000008
:1025400038B50546FFF7E0FF044601462846FFF789
:1025500017FF204638BD0000302383F3118862B690
:1025600070470000002383F3118862B670470000B3
:10257000012070477047000010B4134602681468C9
:102580000022A4465DF8044B6047000000F580502F
:1025900090F859047047000000F5805090F85204FC
:1025A0007047000000F5805090F958047047000013
:1025B0004E20704700F5805208B5FFF7CDFFD2F8E6
:1025C0009834D2F894041844D2F890341844D2F8CD
:1025D00078341844D2F888341844D2F88434184433
:1025E000FFF7C0FF08BD00002DE9F04F0C4600F5D5
:1025F000805185B01F4691F8523405469046BDF88B
:1026000038909BB1D1F874340133C1F87434236825
:102610009A0006D4237B082B0BD9627B0AB10F2BBF
:1026200007D9D1F878340133C1F878344FF0FF304E
:102630000FE0FFF791FFEB6AD3F8C42012F4001A01
:102640000AD0D1F87C3400200133C1F87C34FFF784
:1026500089FF05B0BDE8F08F22684FF0480BD3F832
:10266000C460002A6B6AC6F30446B4BF42F08042DD
:1026700092041BFB063BCBF8002023685B004FEA6B
:10268000066344BF42F00052CBF80020227B43EAAD
:1026900002437201CBF80430607B18B343F440135B
:1026A000CBF80430D1F8A4340133C1F8A434AB180A
:1026B00003F58353197B41F020011973207B0392AA
:1026C00000F05CFF0330039A80105FFA8AF30AF18E
:1026D000010A83420DDA04EB83010BEB83034968A3
:1026E0009960F2E7AB1803F58353197B60F345114A
:1026F000E3E70121EB6A04F10C00B140C3F8D0100C
:10270000AB18214603F58253C3E9048705EB461352
:1027100003F58253183351F804CB814243F804CBBC
:10272000F9D109882A442846198041F26803D65015
:1027300002F5805209F0030392F86C1043F0100385
:1027400021F01F010B43214682F86C304246FFF70F
:1027500009FF3B46CDF8009000F0D6FE012078E757
:102760002DE9F04700F58056044696F85254002DA6
:1027700040F00181037C032B40F092802B462846D9
:102780002F465FFA83FC944510DA01EBCC0E51F82A
:102790003CC0BCF1000F04DBDEF804C0BCF1000F4C
:1027A00002DB01370133ECE70130FBE7FFF7D4FE32
:1027B000E36AF0B9D3F8800040F00200C3F880006B
:1027C0004E23E06A002F6ED1D0F8803043F0010331
:1027D000C0F88030694B6A4A1B6803F1805303F5E7
:1027E0002C539B009342A36240F2AF80654800F0F7
:1027F00063FE4D2842D8DFF884814FEA004EDFF8AF
:102800008891D8F800C04EEA8C0EC3F884E00CF131
:10281000805303F52C539B00636100EB0C03D4F849
:102820002CC0C8F80030C0F14E03DCF8800040F046
:102830003000CCF880004FF0000CD4F81480E6464D
:102840005FFA8CF08242BCDD01EBC00A51F8300027
:10285000002810DBDAF804A0BAF1000F0BDA09EA5D
:1028600000400AF07F0A40EA0A0040F0084048F8B9
:102870002E000EF1010E0CF1010CE1E79A6922F035
:1028800001029A6100F01EFE0646E36A9B69D907C1
:1028900004D500F017FE831BFA2BF6D9FFF762FE72
:1028A0002846BDE8F087B7EB530F3DD2DFF8CCE008
:1028B0004FEA074CDEF800304CEA830CC0F888C0C1
:1028C00003F1805003EB4703002700F52C50CEF8AE
:1028D0000030BC468000A061E06AD0F8803043F050
:1028E0000C03C0F88030D4F818E0FBB29A427FF7AE
:1028F00071AF51F8330001EBC3080028D8F8043059
:1029000001DB002B0EDB20F0604023F0604340F041
:10291000005043F000434EF83C000EEBCC000CF1AD
:10292000010C43600137E0E7836923F00103836111
:1029300000F0C8FD0646E36A9B69DA07AED500F0F1
:10294000C1FD831BFA2BF6D9A8E7E26A936923F04D
:102950000103936100F0B6FD0746E36A9B69DB075C
:1029600005D500F0AFFDC31BFA2BF6D996E701257C
:1029700086F8525492E7002592E700BF784E002077
:10298000FCB50040F87700080000FF0713B500F51C
:1029900080540191606CFFF7D9FC1F280AD92022CE
:1029A0000199606CFFF748FDA0F12003584258419F
:1029B00002B010BD0020FBE700F5805008B5FFF71E
:1029C000CBFD406CFFF796FCBDE80840FFF7CABDA1
:1029D00000220260828142608260704700220023F0
:1029E00010B5C0E90023002304460C3020F8043C55
:1029F000FFF7EEFF204610BD2DE9F047074688B0EF
:102A00009A46884607F5805468469146FFF7A4FD2C
:102A1000FFF7E4FF606CFFF77FFC1F282DD9202211
:102A20006946606CFFF78CFD202826D194F852345B
:102A30001BB303AD444605AB2E46083403CE9E427D
:102A400044F8080C44F8041C3546F5D1306841467A
:102A500020603846B388A380DDE90023C9E900235C
:102A6000BDF808304A46AAF80030FFF77BFD534610
:102A700008B0BDE8F04700F035BD0020FFF772FD5B
:102A800008B0BDE8F08700002DE9F84F00230646A6
:102A900000F58154054688461034C0E90133264BC1
:102AA00046F8303B374638462037FFF797FFA742B6
:102AB000F9D105F580544FF4805305F5A3594FF033
:102AC000000A26630026676405F5835709F110099B
:102AD0004FF0000B1037E663C4E90D36012384F88C
:102AE000403084F84830A7F11800203747E910AB90
:102AF000FFF76EFF47F8286C4F45F4D184F85884EF
:102B0000A4F85A64A4F85C64A4F85E6484F8606471
:102B1000A4F86264A4F86464A4F8666484F8686441
:102B2000B8F1000F02D0054800F0C6FC044B28465F
:102B3000EB62BDE8F88F00BF387800081C78000809
:102B400000A00040044B10B5197804464A1C1A70C6
:102B5000FFF79AFF204610BD754E00202DE9F04783
:102B600000295FD0304F3148B7FBF1F581428CBF6F
:102B70000A201120431EB5FBF0FC00FB1C50DCB208
:102B800020B1022B1846F5D8002037E00CF1FF35B4
:102B9000B5F5806F32D2C4EBC4094FF47A7009F1F5
:102BA00003034FEAE308C3F3C70308F1010AA4EBE8
:102BB000030E08FB00085FFA8EF65AFA8EFEB8FB89
:102BC000FEFEBEF5617F1BDC1FFA8EF4581C56FA20
:102BD00080F00CFB00FCB7FBFCFC6145D4D1013B51
:102BE000DBB20F2BD0D8711E0020C9B2072905D83F
:102BF000107101201480558053719171BDE8F087E8
:102C000009F1FF334FEAE30EC3F3C7030EF10108E6
:102C1000E41A0EFB0000E6B258FA84F4B0FBF4F4B8
:102C2000A4B2D3E70846E9E700B4C4043F420F006A
:102C300038B540F27772C36A154CC3F8BC2007223E
:102C4000C36AC3F8C8202268C16A930043F4C02352
:102C5000C1F8A03002F1805302F16C01C56A03F59E
:102C60002C53EA3289009B00226041F0E061094A5E
:102C7000C361C5F8C01003F5D87103F56A734162EA
:102C80009342836202D9044800F016FC38BD00BFAD
:102C9000784E0020FCB50040F87700082DE9F04F91
:102CA00000F58055994689B0044695F858348A460F
:102CB0009046012B04D90027384609B0BDE8F08FB3
:102CC000934A52F8231009B942F823009149C4F8F5
:102CD0000CA00B7884F81090C3B9FFF73DFC8E4B25
:102CE000D3F8EC2042F48072C3F8EC20D3F894209F
:102CF00042F48072C3F89420D3F8942022F48072B6
:102D0000C3F8942001230B70FFF72CFC95F8513485
:102D100073B903211320FFF71FFC01F02BFD0321E2
:102D2000152001F027FD012385F85134FFF71AFC27
:102D3000FFF712FCE26A936923F01003936100F03D
:102D4000C1FB0746E36A9E6916F0080607D000F04B
:102D5000B9FBC31BFA2BF5D9FFF704FCABE79A6963
:102D600042F001029A6100F0ADFB0746E36A9A69FE
:102D7000D00705D400F0A6FBC31BFA2BF6D9EBE76E
:102D80009A69002704F5825B42F002020BF1100BF6
:102D90009A61E36A5F65FFF7E5FB686CFFF7AAFAE3
:102DA000202200216846FEF773FF02A8FFF710FEFD
:102DB0006A460BEB06030DF1180E0697944608338E
:102DC000BCE80300F44543F8080C43F8041C6246D1
:102DD000F4D1DCF8000020361860B6F5806F9CF85E
:102DE00004201A71DCD1002304F5A252514620467A
:102DF0001A3285F8503485F85334FFF7AFFE074692
:102E000090B9E26A936923F00103936100F05AFBE1
:102E10000546E36A9B69D9077FF54DAF00F052FB89
:102E2000431BFA2BF5D946E795F85F6495F85E24C5
:102E30003602C5F86CA4E36A46EA426695F8602457
:102E40001643B5F85C2446EA0246DE61B8F1000F8D
:102E500029D004F5A352414620460232FFF77EFEF8
:102E600090B9E26A936923F00103936100F02AFBB1
:102E70000546E36A9B69DA077FF51DAF00F022FB88
:102E8000431BFA2BF5D916E795F8683495F86714C3
:102E90001B01C5F87084E26A43EA0123B5F86414A3
:102EA00043EA0143D360E36A00262046C3F8BC60CE
:102EB000FFF7BEFE85F859646FF04042E36A1A6579
:102EC000164AE36A5A654FF00222E36A9A654FF0A8
:102ED000FF32E36AC3F8E0200322E36A9145DA6532
:102EE0003FF4EAAEE26A936923F00103936100F0D4
:102EF000E9FA0646E36A9B69DB0705D500F0E2FACA
:102F0000831BFA2BF6D9D6E6012385F85234D3E693
:102F1000704E0020744E00200044025855020002FA
:102F20002DE9F04F054689B090469946002741F2B9
:102F3000680A00F58056EB6AD3F8D830FB40D80712
:102F40004AD505EB47124FEA471B5244137919073C
:102F500042D4D6F880340133C6F8803413799A0607
:102F600005EB0B0248BFD6F8A834524444BF0133E6
:102F7000C6F8A834137943F008031371DB0723D58F
:102F800096F8533403B305F582546846FFF726FDDF
:102F900003AB18345C4404F1080C2068083454F87E
:102FA000041C1A46644503C21346F6D120686946DC
:102FB00010602846A2889A800123ADF808302B685B
:102FC000CDE90089DB6B9847D6F8543423B1D6F8A5
:102FD0009C340133C6F89C340137202FABD109B0A3
:102FE000BDE8F08F2DE9F04F0F468DB0044600F09C
:102FF0006BFA82468946002F5BD1E36AD3F8A020A2
:1030000012F4FE0F03D100200DB0BDE8F08FD3F80D
:10301000A420920141BF04F58051D1F894240132DB
:10302000C1F89424D3F8A4205606ECD0D3F8A450C9
:10303000E669C5F305254823E8464FF0000B03FB7E
:1030400005664046FFF7C4FC326851004ABF22F0D3
:103050006043C2F38A4343F00043920048BF43F009
:1030600080430093736813F400131BBF012304F51E
:1030700080528DF80D308DF80D301EBFD2F8AC3473
:103080000133C2F8AC34F38803F00F038DF80C3031
:103090009DF80C0000F072FA5FFA8BF3984225D984
:1030A000F2180CA90BF1010B127A0B4403F82C2C2B
:1030B000EEE7012FA7D1E36AD3F8B02012F4FE0F98
:1030C000A1D0D3F8B420950141BF04F58051D1F8C7
:1030D00094240132C1F89424D3F8B420500692D03D
:1030E000D3F8B450266AC5F30525A4E7EFB9E36A1F
:1030F000C3F8A85004A807ADFFF770FC98E80F00CC
:1031000007C52B800023204604A9ADF8183023689A
:1031100004F58054DB6BCDE904A9984758B1D4F885
:103120008C340133C4F88C346EE7012FE2D1E36AAA
:10313000C3F8B850DEE7D4F8903401200133C4F866
:10314000903461E7F8B505460F4600F58054012636
:1031500039462846FFF746FF10B184F85364F7E775
:10316000D4F8543423B1D4F89C340133C4F89C34DB
:10317000F8BD0000C36AF0B51A6C12F47F0F2BD0B3
:103180001B6C00F5805441F268054FF0010CC4F847
:10319000A0340023471900EB43125E012A44117941
:1031A00011F0020F15D0490713D4B959C66A0CFAA9
:1031B00001F1D6F8CCE011EA0E0F0AD0C6F8D4100F
:1031C000117941F004011171D4F888240132C4F856
:1031D00088240133202BDED1F0BD000010B5264C31
:1031E000264B22680AB340B31A6D92050FD54FF4EF
:1031F00000721A6500F068F950EA01020B4602D02D
:10320000013861F1000302462068FFF789FE1B4A7E
:10321000136D9B012AD523684FF0007103F580538D
:103220001165012283F8592420E001221A65102239
:103230001A654FF480521A6510BD196DC80702D483
:10324000196D490705D50521104619650021FFF7BD
:1032500079FF0A4B1A6DD00602D41A6D510605D5B6
:10326000502201211A652068FFF76CFF2068BDE835
:103270001040FFF77FBF00BF704E002000A000404D
:1032800008B5FFF769F9FFF775FFBDE80840FFF7DC
:1032900069B90000C36AD3F8C00010F07C5005D0B3
:1032A000D3F8C40080F40010C0F340507047000011
:1032B00000F5805008B5FFF74FF9406CFFF72CF888
:1032C000FFF750F943090CBF0120002008BD0000A2
:1032D00000F5805393F8592462B1C16A8A6922F0DB
:1032E00001028A61D3F898240132C3F8982400229D
:1032F00083F85924704700002DE9F74300F5825107
:1033000098460025FFF728F9103141F2680E4FF07A
:10331000010900F5805C00EB4514744423795E07D5
:103320001CD4DB061AD58E69C36A09FA06F6D3F8EF
:10333000CC703E4212D04F6801970F689742019FB0
:1033400077EB08070AD2C3F8D460237943F004036B
:103350002371DCF884340133CCF884340135203116
:10336000202DD8D103B0BDE8F043FFF7FBB8000033
:10337000F8B51E4600230F46054613701446FFF7A6
:1033800097FF80F0010038701EB12846FFF782FFDA
:103390002070F8BD2DE9F04F85B099460D46804666
:1033A000164691F800B0DDE90EA30293137801935D
:1033B00000F08AF82B7804460F4613B93378002BB7
:1033C00042D022463B464046FFF796FFFFF758FFA4
:1033D000FFF77EFF4B4632462946FFF7C9FF2B78A1
:1033E00033B1BBF1000F03D0012005B0BDE8F08F71
:1033F000337813B1019B002BF6D108F5805303936A
:103400005445029B77EB03031ED2039BD3F854046D
:10341000D0B10368AAEB0401DB6889B298474B4638
:10342000324629464046FFF7A3FF2B7813B1BBF184
:10343000000FD9D1337813B1019B002BD4D100F008
:1034400043F804460F46DBE70020CEE708B500202E
:10345000FFF7C4FEBDE8084001F056B808B50120EA
:10346000FFF7BCFEBDE8084001F04EB800B59BB0C8
:10347000EFF3098168226846FEF7E4FBEFF305836A
:10348000014B9B6BFEE700BF00ED00E008B5FFF7C6
:10349000EDFF000000B59BB0EFF30981682268469C
:1034A000FEF7D0FBEFF30583014B5B6BFEE700BF3C
:1034B00000ED00E0FEE700000FB408B5029802F04E
:1034C0001FF8FEE702F0C4BC02F09CBC13B56C46CA
:1034D000031D84E8060094E8030083E8050001204A
:1034E00002B010BD73B58568019155B11B885B07AB
:1034F00007D4D0E900369B6B9847019AC1B2304699
:10350000A847012002B070BDF0B5866889B00546B5
:103510000C465EB1BDF838305B070AD4D0E90037FD
:103520009B6B98472246C1B23846B047012009B08C
:10353000F0BD0022002301F10806CDE9002300239D
:103540000A46ADF8083003AB1068083252F8041C84
:103550001C46B24203C42346F6D11068206092880C
:10356000A280FFF7B1FF0423ADF808302B68CDE946
:103570000001DB6B694628469847D7E7082817D92A
:1035800009280CD00A280CD00B280CD00C280CD001
:103590000D280CD00E2814BF4020302070470C207E
:1035A0007047102070471420704718207047202063
:1035B000704700002DE9F041456A15B94162BDE848
:1035C000F0814B68AC4623F06047C3F38A464FEA6C
:1035D000D37EC3F3807816EA230638BF3E462B46D7
:1035E0005A68BEEBD27F22F060440AD0002A18DA73
:1035F000A40CB44217D19D420FD10D60DEE71346F3
:10360000EEE7A74207D102F08044C2F38072424540
:103610000BD054B1EFE708D2EDE7CCF800100B6007
:10362000CDE7B44201D0B442E5D81A689C46002ADE
:10363000E5D11960C3E700002DE9F047089D01F0CE
:10364000070400EBD1004FF47F494FEAD50822442C
:1036500005F00705944201D1BDE8F08704F00707A3
:1036600005F0070A111B08EBD50E57453E4613F827
:103670000EC038BF5646C6F108068E4228BF0E4619
:10368000E108415C34443544B94029FA06F721FA8F
:103690000AF1FFB28CEA010147FA0AF739408CEAD5
:1036A000010C03F80EC0D5E780EA0120082341F29F
:1036B000210201B2013B4000002980B2B8BF504056
:1036C00013F0FF03F5D1704738B50C468D18A542AD
:1036D00000D138BD14F8011BFFF7E6FFF7E7000043
:1036E00042684AB1136881894360438901339BB2C0
:1036F0009942438138BF83811046704770B588B0C6
:10370000044620220D4668460021FEF7C1FA2046F5
:103710000495FFF7E5FF024660B16B46054608AE2B
:103720001C46083503CCB44245F8080C45F8041C87
:103730002346F5D1104608B070BD0000082817D9FF
:1037400009280CD00A280CD00B280CD00C280CD03F
:103750000D280CD00E2814BF4020302070470C20BC
:1037600070471020704714207047182070472020A1
:1037700070470000082817D90C280CD910280CD93C
:1037800014280CD918280CD920280CD930288CBF23
:103790000F200E207047092070470A2070470B2029
:1037A00070470C2070470D20704700002DE9F8434A
:1037B000078C0446072F1ED900254FF6FF73D0E96A
:1037C0000298C5F12006A5F1200029FA05F1083577
:1037D00008FA06F628FA00F0314301431846C9B248
:1037E000FFF762FF402D0346EBD13A46E169BDE8A1
:1037F000F843FFF769BF4FF6FF70BDE8F88300009C
:1038000010B54B6823B9CA8A63F30902CA8210BD96
:1038100004691A681C600361C38A013BC3824A6061
:10382000EFE700002DE9F84F1D46CB8A0F46814691
:10383000C3F30901924605290B4630D00020AAB2F5
:1038400007F11A049EB21FFA80F8042E0FD8904593
:1038500003F1010306D30A44FB8A62F30903012042
:10386000FB821AE01AF800600130E654EAE790455E
:10387000F1D2A1F1050B1C237C68BBFBF3F203FB27
:1038800012BB1FFA8BF6002C45D14846FFF728FFE4
:10389000044638B978606FF00200BDE8F88F4FF049
:1038A0000008E6E7002606607860ADB24FF0000B36
:1038B000454510D90AEB0803221D13F8011B08F136
:1038C00001089155B1B21FFA88F81B292BD0454544
:1038D00006F10106F1D8FB8AC3F30902154465F32A
:1038E0000903BCE701321C4692B22368002BF9D1D0
:1038F0006B1F0B441C21B3FBF1F301339BB29A42C3
:10390000D3D2BBF1000FD0D14846FFF7E9FE20B972
:10391000C4F800B0BFE70122E7E7C0F800B05E4698
:1039200020600446C1E74545D5D94846FFF7D8FE93
:1039300008B92060AFE7C0F800B000262060044658
:10394000B6E700002DE9F04F1C46074688462DEDEE
:10395000028B83B05B690192002B00F09A80238C6C
:103960002BB1E269002A00F09480072B35D807F1CB
:103970000C00FFF7B5FE054638B96FF00205284682
:1039800003B0BDEC028BBDE8F08F14220021FEF7DE
:103990007FF9228CE16905F10800FEF753F9208CCC
:1039A00048F00041013080B2FFF7E4FEFFF7C6FEA9
:1039B000013880B220840130287438466369228C33
:1039C0001B782A4403F01F0363F03F0313726960FE
:1039D0002946FFF7EFFD0125D1E74FF0000900F17F
:1039E0000C034FF0800A4E464D4608EE103A18EE92
:1039F000100AFFF775FE83460028BED0142200216E
:103A0000FEF746F9002E3AD1019B0222ABF80830AE
:103A10000BF1080E1FFA82FC218C0CF10100BCF1A5
:103A2000060F80B201D88E422BD3FFF7A3FE8E4241
:103A300008BF4FF0400AFFF781FE62690138013587
:103A400012781BFA80F1013002F01F022DB242EA17
:103A5000491289F001094AEA020A48F0004281F855
:103A600008A059468BF810003846CBF804204FF0D8
:103A7000000AFFF79FFD238CB342B8D17FE70022F5
:103A8000C6E7E169895D01360EF80210B6B201326F
:103A9000C0E76FF0010572E7F8B515460E46302213
:103AA000002104461F46FEF7F3F8069BB5F5001FFC
:103AB000A760636004F11000079B34BF6A094FF6EA
:103AC000FF72E661A362002397B29A4206D80023F0
:103AD0000360A782E3822383E360F8BD06600133BD
:103AE00030462036F1E7000003781BB94BB2002BBB
:103AF000C8BF01707047000000787047F8B50C46E9
:103B0000C969074611B9238C002B37D1257E1F2D9B
:103B100034D8387828BB228C072A2CD8268A36F04D
:103B200003032BD14FF6FF70FFF7CEFD20F001000D
:103B300031024FF6FF72400441EA0561400C41EA50
:103B40004025234629463846FFF7FCFE002807DDBE
:103B5000626913780133DBB21F2B88BF0023137017
:103B6000F8BD218A2D0645EA012505432046FFF7C9
:103B70001DFE0246E5E76FF00300F1E76FF001007C
:103B8000EEE7000070B58AB00446164600212822F0
:103B900068461D46FEF77CF8BDF838306946204679
:103BA000ADF810300F9B05939DF840308DF818301C
:103BB000119B0793BDF84830CDE90265ADF8203080
:103BC000FFF79CFF0AB070BD2DE9F041D3690546AF
:103BD0000C4616460BB9138C5BBB377E1F2F28D8BB
:103BE00095F80080B8F1000F26D03046FFF7DEFDD3
:103BF000337821020246284641EAC331338A41EA3A
:103C0000080141EA076141EA0341334641F080017E
:103C1000FFF798FE00280ADD3378012B07D172697F
:103C200013780133DBB21F2B88BF00231370BDE86C
:103C3000F0816FF00100FAE76FF00300F7E7000092
:103C4000F0B58BB004460D46174600212822684681
:103C50001E46FEF71DF89DF84C30294620465A1E98
:103C6000534253416A468DF800309DF84030ADF81C
:103C70001030119B05939DF848308DF81830149B37
:103C80000793BDF85430CDE90276ADF82030FFF748
:103C90009BFF0BB0F0BD0000406A00B104307047DC
:103CA000436A1A68426202691A600361C38A013B6F
:103CB000C38270472DE9F041D0F8208014461D469C
:103CC000184E4146002709B9BDE8F081D1E9022329
:103CD000A21A65EB0303964277EB03031ED2036A35
:103CE0008B420DD1FFF78CFD036A1B6803620369E9
:103CF0000B60C38A0161013B016AC3828846E2E727
:103D0000FFF77EFD0B68C8F8003003690B60C38ABB
:103D10000161013BC382D8F80010D4E788460968E6
:103D2000D1E700BF80841E002DE9F04F8BB00D4617
:103D300014469B46DDF850908046002800F018811C
:103D4000B9F1000F00F01481531E3F2B00F21081D7
:103D5000012A03D1BBF1000F40F00A810023CDE915
:103D60000833B8F81430B5EBC30F4FEAC30703D3D9
:103D700000200BB0BDE8F08F2B199F42D8F80C3013
:103D800036BF7F1B2746FFB21BB9D8F81030002B77
:103D90007AD0272D4DD8C5F1280600232946B742F1
:103DA000009308ABD8F808002CBFF6B23E46A7EB4C
:103DB000060A354432465FFA8AFAFFF73DFCB8F846
:103DC0001430282103F10053053BDB000493D8F89D
:103DD0000C300393039B13B1BAF1000F2CD1D8F828
:103DE000100040B1BAF1000F05D008AB5246691A75
:103DF0000096FFF721FC38B2002FB9D066070AD031
:103E00000AAB624203EBD40102F0070211F8083C4E
:103E1000134101F8083C082C3DD9102C40F2B58024
:103E2000202C40F2B780BBF1000F00F09C800823EB
:103E300035E0BA460026C2E7049BE02B28BFE0230A
:103E400006930B44AB42059315D95A1B0398691A84
:103E50000096924508AB00F1040034BF5246D2B23E
:103E60000792FFF7E9FB079A1644AAEB020A1544EA
:103E7000F6B25FFA8AFA049B069A05999B1A049394
:103E8000039B1B680393A5E700933A4608AB2946BA
:103E9000D8F80800ADE7BBF1000F13D00123B4EB55
:103EA000C30F6BD0082C12D89DF82030621E23FA65
:103EB00002F2D50706D54FF0FF3202FA04F423438D
:103EC0008DF820309DF8203089F8003051E7102C13
:103ED00012D8BDF82030621E23FA02F2D10706D5AF
:103EE0004FF0FF3202FA04F42343ADF82030BDF85E
:103EF0002030A9F800303CE7202C0FD80899631E29
:103F000021FA03F3DA0705D54FF0FF3202FA04F481
:103F10000C430894089BC9F800302AE7402C2AD0AB
:103F2000611EC4F12102A4F12103DDE9086526FA2E
:103F300001F105FA02F225FA03F311431943CB0705
:103F400011D50122A4F12003C4F1200102FA03F3E8
:103F500022FA01F1A2400B43524263EB4303324386
:103F60002B43CDE90823DDE90823C9E9002300E755
:103F70006FF00100FDE66FF00800FAE6082CA1D909
:103F8000102CB4D9202CEED8C4E7BBF1000FAED072
:103F9000022384E7BBF1000FBCD004237FE70000BD
:103FA000012A30B5144638BF012485B00025402CC5
:103FB00028BF4024012ACDE9025518D81B788DF876
:103FC000083063070AD004AB624203EBD40502F069
:103FD000070215F8083C934005F8083C0346009199
:103FE0002246002102A8FFF727FB05B030BD082AB2
:103FF000E4D9102A03D81B88ADF80830E1E7202A5D
:1040000095BF1B68D3E900230293CDE90223D8E7CB
:1040100010B5CB681BB98B600B618B8210BD046936
:104020001A681C600361C38A013BC382CA60F0E75F
:1040300003064CBFC0F3C0300220704708B50246EB
:10404000FFF7F6FF022806D15306C2F30F2001D175
:1040500000F0030008BDC2F30740FBE72DE9F04F75
:1040600093B004460D46CDE903230A681046FFF7D6
:10407000DFFF0228824614BFC2F306260026002A6C
:1040800080F2F38112F0C04940F0EF81097B0029F2
:1040900000F0EB81022803D02378B34240F0E8819E
:1040A000C2F3046310462944069302F07F0305938C
:1040B000FFF7C4FF059B002283464FEA8348002395
:1040C00048EA0A4848EA4668CE78CDE90823F30969
:1040D00048EA0008029368D0059B024608A92046DA
:1040E000009353466768B847002800F0C481276AE8
:1040F0004FB9414604F10C00FFF700FB074690B9A9
:104100006FF0020055E03B6998450DD03F68002FE5
:10411000F9D1414604F10C00FFF7F0FA07460028F8
:10412000EED0236A3B60276297F817C006F01F089D
:10413000CCF3840CACEB0800A8EB0C031FFA80FE58
:104140000028B8BF0EF120001FFA83FEB8BF00B2EE
:10415000002B0793B8BF0EF12003D7E90221BCBFA3
:104160001BB2079352EA010338D0039B4FF0000CB7
:10417000DFF820E39A1A049B63EB010196457CEB80
:1041800001032BD36B7B97F81AE0734519D1029B7F
:10419000002B78D0012821DC7868F8B9DFF8F0C26C
:1041A000944570EB010316D337E0276A27B96FF007
:1041B0000C0013B0BDE8F08F3B699845B4D03F6860
:1041C000F4E7B34890427CEB010301D30020F0E711
:1041D000029B002BFAD0079B0F2B17DCFA7DB30054
:1041E0003946204602F0030203F07C031343FB75BB
:1041F000FFF706FB6B7BBB76029B3BB9FB7DC3F3F2
:104200008402013262F38603FB75D0E76A7BBB7ED2
:104210009A42DBD1029B002B35D0B309022B32D05E
:10422000039B142200210DA8BB60049BFB60FDF7DB
:104230002FFD039B0AA920460A93049BADF83EB0CC
:104240000B932B1D8DF840A00C932B7B8DF8418098
:10425000013BDBB2ADF83C30069B8DF84230059B4C
:104260008DF8433094F82C3083F001038DF84430FE
:10427000A3689847FB7DC3F38403013303F01F0356
:104280009B02FB82A2E7FB7DC6F34012B2EBD31F79
:1042900040F0F480C3F38403434540F0F280029A77
:1042A000B6092B7B002A4DD0F2075DD4032B40F2D8
:1042B000EB80039BAE1D394604F10C00BB60324617
:1042C000049BFB602B7B033BDBB2FFF7ABFA0028C0
:1042D0000CDA39462046FFF793FAFB7DC3F38403DB
:1042E000013303F01F039B02FB8209E7AB88DDE982
:1042F00008843B834FF6FF73C9F12000A9F1200227
:1043000028FA09F109F1080904FA00F024FA02F286
:10431000014318461143C9B2FFF7C6F9B9F1400F7E
:104320000346E9D1B88231462A7B033AD2B2FFF77D
:10433000CBF9FB7DB882DA43C2F3C01262F3C71334
:10434000FB7543E786B92E1D013B394604F10C008D
:10435000DBB23246FFF766FA0028BADB2A7B314629
:10436000B88A013AD2B2E2E7F98A013BC1F3090106
:10437000DAB204295BD8281D002307F11B069A42F4
:1043800008D910F801CB013306F801C00131DBB2C6
:104390000529F4D1039993420A9138BF0433049953
:1043A0002CBF002355FA83F30B9107F11B010C91ED
:1043B00079680E930D91291DFB8AADF83EB0C3F3C9
:1043C00009038DF840A08DF841801A44069B8DF8B2
:1043D0004230059BADF83C208DF8433094F82C30EA
:1043E00083F001038DF844300023B88A7B602A7B78
:1043F000013AFFF769F93B8BB882834203D1A36886
:104400000AA92046984720460AA9FFF701FEFB7D2E
:10441000BA8AC3F38403013303F01F039B02FB82B8
:104420003B8B9A420CBF00206FF01000C1E67B6806
:10443000002BAFD0052001E01C3033461E68002E53
:10444000FAD1091A2E1D081D184401EB090C5FFA58
:1044500089F3BCF11B0F9DD89A429BD916F8013BFA
:1044600009F1010900F8013BEFE76FF00900A0E650
:104470006FF00A009DE66FF00B009AE66FF00D00FA
:1044800097E66FF00E0094E66FF00F0091E600BF24
:1044900040420F0080841E00EFF309830549683312
:1044A0004A6B22F001024A6383F30988002383F3F5
:1044B0001188704700EF00E0302080F3118862B669
:1044C0000D4B0E4AD96821F4E0610904090C0A4336
:1044D0000B49DA60D3F8FC2042F08072C3F8FC206C
:1044E000084AC2F8B01F116841F001011160202292
:1044F000DA7783F82200704700ED00E00003FA0548
:1045000055CEACC5001000E0302310B583F3118800
:104510000E4B5B6813F4006314D0F1EE103AEFF326
:1045200009844FF08073683CE361094BDB6B2366C1
:1045300084F3098800F0A2FF10B1064BA36110BDFF
:10454000054BFBE783F31188F9E700BF00ED00E0BE
:1045500000EF00E0430700084607000802684368D0
:104560001143016003B1184770470000024A136805
:1045700043F0C003136070470078004013B50E4C41
:10458000204600F0A1FA04F1140000234FF4007259
:104590000A49009400F05EF9094B4FF40072094992
:1045A00004F13800009400F0D7F9074A074BC4E93A
:1045B000172302B010BD00BF804E0020EC4E00203B
:1045C0006D450008EC5000200078004000E1F50542
:1045D000037C30B5214C002918BF0C46012B0CD1AF
:1045E0001F4B984209D11F4B9A6C42F080429A644B
:1045F0001A6F42F080421A671B6F2268036EC16D0A
:1046000003EB52038466B3FBF2F36268150442BF06
:1046100023F0070503F0070343EA4503CB60A368D3
:1046200043F040034B60E36843F001038B6042F4C6
:10463000967343F001030B604FF0FF330B6251059B
:1046400005D512F0102205D0B2F1805F04D080F8B9
:10465000643030BD7F23FAE73F23F8E7787800081D
:10466000804E0020004502582DE9F047C66D0546F2
:104670003768F469210734621AD014F0080118BFB2
:104680004FF48071E20748BF41F02001A3074FF0CB
:10469000300348BF41F04001600748BF41F080014E
:1046A00083F31188281DFFF759FF002383F3118836
:1046B000E2050AD5302383F311884FF48061281D69
:1046C000FFF74CFF002383F311884FF030094FF0C0
:1046D000000A14F0200838D13B0616D54FF03009F7
:1046E00005F1380A200610D589F31188504600F0EC
:1046F00067F9002836DA0821281DFFF72FFF27F079
:1047000080033360002383F31188790614D5620691
:1047100012D5302383F31188D5E913239A4208D1A7
:104720002B6C33B127F040071021281DFFF716FF2F
:104730003760002383F31188E30618D5AA6E136946
:10474000ABB15069BDE8F047184789F31188736A27
:10475000284695F86410194000F0D0F98AF31188C2
:10476000F469B6E7B06288F31188F469BAE7BDE886
:10477000F0870000090100F16043012203F5614365
:10478000C9B283F8001300F01F039A4043099B004D
:1047900003F1604303F56143C3F880211A60704759
:1047A000F8B51546826804460B46AA4200D28568D1
:1047B000A1692669761AB5420BD218462A46FDF73A
:1047C00041FAA3692B44A3612846A3685B1BA3603D
:1047D000F8BD0CD9AF1B18463246FDF733FA3A46FE
:1047E000E1683044FDF72EFAE3683B44EBE71846F6
:1047F0002A46FDF727FAE368E5E70000836893425D
:10480000F7B50446154600D28568D4E90460361A27
:10481000B5420BD22A46FDF715FA63692B44636152
:104820002846A3685B1BA36003B0F0BD0DD93246D8
:10483000AF1B0191FDF706FA01993A46E068314451
:10484000FDF700FAE3683B44E9E72A46FDF7FAF989
:10485000E368E4E710B50A440024C361029B846066
:10486000C16002610362C0E90000C0E9051110BD2A
:1048700008B5D0E90532934201D1826882B98268D5
:10488000013282605A1C426119700021D0E9043261
:104890009A4224BFC368436100F0C2FE002008BDF5
:1048A0004FF0FF30FBE7000070B5302304460E46A2
:1048B00083F31188A568A5B1A368A269013BA36031
:1048C000531CA36115782269934224BFE368A36156
:1048D000E3690BB120469847002383F311882846EB
:1048E00007E03146204600F08BFE0028E2DA85F32F
:1048F000118870BD2DE9F74F04460E4617469846BD
:10490000D0F81C904FF0300A8AF311884FF0000B5A
:10491000154665B12A4631462046FFF741FF03465A
:1049200060B94146204600F06BFE0028F1D000231C
:1049300083F31188781B03B0BDE8F08FB9F1000F45
:1049400003D001902046C847019B8BF31188ED1AD4
:104950001E448AF31188DCE7C160C361009B82605A
:104960000362C0E905111144C0E90000016170470C
:10497000F8B504460D461646302383F31188A76820
:10498000A7B1A368013BA36063695A1C62611D70F3
:10499000D4E904329A4224BFE3686361E3690BB14E
:1049A00020469847002080F3118807E031462046D2
:1049B00000F026FE0028E2DA87F31188F8BD000037
:1049C000D0E9052310B59A4201D182687AB982688C
:1049D0000021013282605A1C82611C7803699A426C
:1049E00024BFC368836100F01BFE204610BD4FF05A
:1049F000FF30FBE72DE9F74F04460E461746984671
:104A0000D0F81C904FF0300A8AF311884FF0000B59
:104A1000154665B12A4631462046FFF7EFFE0346AC
:104A200060B94146204600F0EBFD0028F1D000239C
:104A300083F31188781B03B0BDE8F08FB9F1000F44
:104A400003D001902046C847019B8BF31188ED1AD3
:104A50001E448AF31188DCE7026843681143016051
:104A600003B11847704700001430FFF743BF000040
:104A70004FF0FF331430FFF73DBF00003830FFF731
:104A8000B9BF00004FF0FF333830FFF7B3BF00006D
:104A90001430FFF709BF00004FF0FF311430FFF76B
:104AA00003BF00003830FFF763BF00004FF0FF3254
:104AB0003830FFF75DBF0000012914BF6FF013000D
:104AC00000207047FFF75ABD044B0360002343608A
:104AD000C0E9023301230374704700BF90780008D7
:104AE00010B53023044683F31188FFF771FD0223CC
:104AF0000020237480F3118810BD000038B5C3690D
:104B000004460D461BB904210844FFF7A5FF2946BA
:104B100004F11400FFF7ACFE002806DA201D4FF464
:104B20000061BDE83840FFF797BF38BD02684368B1
:104B30001143016003B118477047000013B5406B83
:104B400000F58054D4F8A4381A681178042914D1D7
:104B5000017C022911D11979012312898B4013425A
:104B60000BD101A94C3002F00BF9D4F8A44802464D
:104B7000019B2179206800F0DFF902B010BD000030
:104B8000143002F08DB800004FF0FF33143002F003
:104B900087B800004C3002F05FB900004FF0FF33DF
:104BA0004C3002F059B90000143002F05BB800003C
:104BB0004FF0FF31143002F055B800004C3002F0D5
:104BC0002BB900004FF0FF324C3002F025B9000045
:104BD0000020704710B500F58054D4F8A4381A6846
:104BE0001178042917D1017C022914D159790123A4
:104BF00052898B4013420ED1143001F0EDFF024672
:104C000048B1D4F8A4484FF4407361792068BDE8F6
:104C1000104000F07FB910BD406BFFF7DBBF000014
:104C2000704700007FB5124B01250426044603603F
:104C30000023057400F1840243602946C0E9023371
:104C40000C4B0290143001934FF44073009601F026
:104C50009FFF094B04F69442294604F14C0002944C
:104C6000CDE900634FF4407302F066F804B070BD04
:104C7000B8780008194C00083D4B00080A6830233A
:104C800083F311880B790B3342F823004B791333EC
:104C900042F823008B7913B10B3342F8230000F55F
:104CA0008053C3F8A41802230374002080F31188F2
:104CB0007047000038B5037F044613B190F85430B4
:104CC000ABB90125201D0221FFF730FF04F11400CC
:104CD0006FF00101257700F0AFFC04F14C0084F87F
:104CE00054506FF00101BDE8384000F0A5BC38BD5C
:104CF00010B5012104460430FFF718FF0023237785
:104D000084F8543010BD000038B504460025143036
:104D100001F056FF04F14C00257702F025F8201D24
:104D200084F854500121FFF701FF2046BDE83840C8
:104D3000FFF750BF90F8803003F06003202B06D1BE
:104D400090F881200023212A03D81F2A06D80020AA
:104D50007047222AFBD1C0E91D3303E0034A4267B2
:104D600007228267C3670120704700BF3C220020F2
:104D700037B500F58055D5F8A4381A68117804299C
:104D80001AD1017C022917D11979012312898B408C
:104D9000134211D100F14C04204602F0A5F858B19D
:104DA00001A9204601F0ECFFD5F8A4480246019B7A
:104DB0002179206800F0C0F803B030BD01F10B0389
:104DC000F0B550F8236085B004460D46FEB130239F
:104DD00083F3118804EB8507301D0821FFF7A6FE39
:104DE000FB6806F14C005B691B681BB1019001F088
:104DF000D5FF019803A901F0C3FF024648B1039B08
:104E00002946204600F098F8002383F3118805B066
:104E1000F0BDFB685A691268002AF5D01B8A013B75
:104E20001340F1D104F18002EAE70000133138B5F4
:104E300050F82140ECB1302383F3118804F58053FE
:104E4000D3F8A4281368527903EB8203DB689B69CB
:104E50005D6845B104216018FFF768FE294604F13A
:104E6000140001F0C3FE2046FFF7B4FE002383F3D5
:104E7000118838BD7047000001F096B90123402227
:104E8000002110B5044600F8303BFCF701FF002379
:104E9000C4E9013310BD000010B53023044683F38C
:104EA00011882422416000210C30FCF7F1FE2046DD
:104EB00001F09CF902230020237080F3118810BDBB
:104EC00070B500EB8103054650690E461446DA6062
:104ED00018B110220021FCF7DBFEA06918B11022E6
:104EE0000021FCF7D5FE31462846BDE8704001F0B0
:104EF0007DBA000083682022002103F0011310B561
:104F0000044683601030FCF7C3FE2046BDE8104025
:104F100001F0F8BAF0B4012500EB810447898D4017
:104F2000E4683D43A469458123600023A260636077
:104F3000F0BC01F015BB0000F0B4012500EB8104CA
:104F400007898D40E4683D4364690581236000233F
:104F5000A2606360F0BC01F08BBB000070B502235F
:104F600000250446242203702946C0F888500C30DE
:104F700040F8045CFCF78CFE204684F8705001F089
:104F8000C9F963681B6823B129462046BDE8704013
:104F9000184770BD0378052B10B504460AD080F879
:104FA0008C300523037043681B680BB104219847BC
:104FB0000023A36010BD00000178052906D190F8F8
:104FC0008C20436802701B6803B1184770470000CB
:104FD00070B590F87030044613B1002380F870303B
:104FE00004F18002204601F0B1FA63689B68B3B90E
:104FF00094F8803013F0600535D00021204601F090
:10500000A3FD0021204601F093FD63681B6813B1E6
:10501000062120469847062384F8703070BD20464C
:1050200098470028E4D0B4F88630A26F9A4288BF2F
:10503000A36794F98030A56F002B4FF0300380F206
:105040000381002D00F0F280092284F8702083F3A0
:10505000118800212046D4E91D23FFF76DFF0023AE
:1050600083F31188DAE794F8812003F07F0343EAA1
:10507000022340F20232934200F0C58021D8B3F5FA
:10508000807F48D00DD8012B3FD0022B00F09380B9
:10509000002BB2D104F1880262670222A267E367A3
:1050A000C1E7B3F5817F00F09B80B3F5407FA4D1C9
:1050B00094F88230012BA0D1B4F8883043F0020379
:1050C00032E0B3F5006F4DD017D8B3F5A06F31D0F3
:1050D000A3F5C063012B90D86368204694F8822022
:1050E0005E6894F88310B4F88430B047002884D008
:1050F000436863670368A3671AE0B3F5106F36D09F
:1051000040F6024293427FF478AF5C4B6367022320
:10511000A3670023C3E794F88230012B7FF46DAFBF
:10512000B4F8883023F00203A4F88830C4E91D5590
:10513000E56778E7B4F88030B3F5A06F0ED194F846
:105140008230204684F88A3001F042F963681B6897
:1051500013B1012120469847032323700023C4E99B
:105160001D339CE704F18B0363670123C3E72378B6
:10517000042B10D1302383F311882046FFF7BAFEA9
:1051800085F311880321636884F88B5021701B68B4
:105190000BB12046984794F88230002BDED084F87B
:1051A0008B300423237063681B68002BD6D0022148
:1051B00020469847D2E794F8843020461D0603F035
:1051C0000F010AD501F0B4F9012804D002287FF4B8
:1051D00014AF2B4B9AE72B4B98E701F09BF9F3E7C1
:1051E00094F88230002B7FF408AF94F8843013F0E9
:1051F0000F01B3D01A06204602D501F0BDFCADE781
:1052000001F0AEFCAAE794F88230002B7FF4F5AEF3
:1052100094F8843013F00F01A0D01B06204602D56D
:1052200001F092FC9AE701F083FC97E7142284F8DE
:10523000702083F311882B462A4629462046FFF723
:1052400069FE85F31188E9E65DB1152284F87020C6
:1052500083F3118800212046D4E91D23FFF75AFE6D
:10526000FDE60B2284F8702083F311882B462A4632
:1052700029462046FFF760FEE3E700BFE878000814
:10528000E0780008E478000838B590F870300446FB
:10529000002B3ED0063BDAB20F2A34D80F2B32D87F
:1052A000DFE803F037313108223231313131313129
:1052B00031313737856FB0F886309D4214D2C368DC
:1052C0001B8AB5FBF3F203FB12556DB9302383F350
:1052D00011882B462A462946FFF72EFE85F31188B2
:1052E0000A2384F870300EE0142384F870303023E1
:1052F00083F31188002320461A461946FFF70AFE59
:10530000002383F3118838BDC36F03B1984700238E
:10531000E7E70021204601F017FC0021204601F0BC
:1053200007FC63681B6813B10621204698470623D3
:10533000D7E7000010B590F870300446142B29D040
:1053400017D8062B05D001D81BB110BD093B022B85
:10535000FBD80021204601F0F7FB0021204601F098
:10536000E7FB63681B6813B10621204698470623B4
:1053700019E0152BE9D10B2380F87030302383F32B
:10538000118800231A461946FFF7D6FD002383F340
:105390001188DAE7C3689B695B68002BD5D1C36FBE
:1053A00003B19847002384F87030CEE70023826869
:1053B000037503691B6899689142FBD25A680360C0
:1053C000426010605860704700238268037503696B
:1053D0001B6899689142FBD85A680360426010606C
:1053E0005860704708B50846302383F311880B7D59
:1053F000032B05D0042B0DD02BB983F3118808BDE6
:105400008B6900221A604FF0FF338361FFF7CEFFF4
:105410000023F2E7D1E9003213605A60F3E700009D
:10542000FFF7C4BF054BD968087518680268536058
:105430001A600122D8600275FBF76EB9F0520020A5
:105440000C4B30B5DD684B1C87B004460FD02B46A3
:10545000094A684600F084F92046FFF7E3FF009B05
:1054600013B1684600F086F9A86907B030BDFFF7B0
:10547000D9FFF9E7F0520020E5530008044B1A6801
:10548000DB6890689B68984294BF002001207047B9
:10549000F0520020084B10B51C68D8682268536091
:1054A0001A600122DC602275FFF78EFF014620465C
:1054B000BDE81040FBF730B9F0520020044B1A68E9
:1054C000DB6892689B689A4201D9FFF7E3BF704797
:1054D000F052002038B5074C012300250649074843
:1054E0002370656001F03EFD0223237085F311886F
:1054F00038BD00BF58550020F0780008F052002059
:1055000008B572B6044B186500F06AFC00F03CFD6B
:10551000024B03221A70FEE7F0520020585500207B
:1055200000F05EB9EFF3118020B9EFF3058330226C
:1055300082F311887047000010B530B9EFF305848D
:10554000C4F3080414B180F3118810BDFFF7B6FF4F
:1055500084F31188F9E70000034A516853685B1A25
:105560009842FBD8704700BF001000E08B60022318
:10557000086108468B8270478368A3F1840243F870
:10558000142C026943F8442C426943F8402C094A20
:1055900043F8242CC268A3F1200043F8182C0222FF
:1055A00003F80C2C002203F80B2C034A43F8102CB0
:1055B000704700BF31070008F052002008B5FFF720
:1055C000DBFFBDE80840FFF72BBF0000024BDB68A4
:1055D00098610F20FFF726BFF0520020302383F39D
:1055E0001188FFF7F3BF000008B50146302383F3AD
:1055F00011880820FFF724FF002383F3118808BDDA
:10560000064BDB6839B1426818605A60136043602A
:105610000420FFF715BF4FF0FF307047F052002015
:105620000368984206D01A68026050601846996173
:10563000FFF7F6BE7047000038B504460D462068F7
:10564000844200D138BD036823605C608561FFF748
:10565000E7FEF4E7036810B59C68A2420CD85C68CA
:105660008A600B604C602160596099688A1A9A6060
:105670004FF0FF33836010BD121B1B68ECE7000086
:105680000A2938BF0A2170B504460D460A2660195A
:1056900001F060FC01F048FC041BA54203D8751C16
:1056A00004462E46F3E70A2E04D90120BDE87040D7
:1056B00001F098BC70BD0000F8B5144B0D460A2AE5
:1056C0004FF00A07D96103F11001826038BF0A2246
:1056D000416019691446016048601861A81801F01A
:1056E00029FC01F021FC431B0646A34206D37C1C87
:1056F00028192746354601F02DFCF2E70A2F04D978
:105700000120BDE8F84001F06DBCF8BDF05200206A
:10571000F8B506460D4601F007FC0F4A134653F84C
:10572000107F9F4206D12A4601463046BDE8F84028
:10573000FFF7C2BFD169BB68441A2C1928BF2C4699
:10574000A34202D92946FFF79BFF22463146034870
:10575000BDE8F840FFF77EBFF05200200053002064
:10576000C0E90323002310B45DF8044B4361FFF745
:10577000CFBF000010B5194C236998420DD0816845
:10578000D0E9003213605A609A680A449A60002394
:1057900003604FF0FF33A36110BD0268234643F856
:1057A000102F53600022026022699A4203D1BDE8A3
:1057B000104001F0C9BB936881680B44936001F00D
:1057C000B3FB2269E1699268441AA242E4D9114408
:1057D000BDE81040091AFFF753BF00BFF052002088
:1057E0002DE9F047DFF8BC8008F110072C4ED8F8FF
:1057F000105001F099FBD8F81C40AA68031B9A428C
:105800003ED814444FF00009D5E90032C8F81C40D6
:1058100013605A60C5F80090D8F81030B34201D137
:1058200001F092FB89F31188D5E9033128469847A6
:10583000302383F311886B69002BD8D001F074FBFF
:105840006A69A0EB040982464A450DD2022001F0A4
:10585000C9FB0022D8F81030B34208D1514628467F
:10586000BDE8F047FFF728BF121A2244F2E712EB17
:1058700009092946384638BF4A46FFF7EBFEB5E727
:10588000D8F81030B34208D01444C8F81C00211ACC
:10589000A960BDE8F047FFF7F3BEBDE8F08700BFA1
:1058A00000530020F052002000207047FEE7000067
:1058B000704700004FF0FF307047000002290CD005
:1058C000032904D00129074818BF00207047032A84
:1058D00005D8054800EBC200704704487047002017
:1058E000704700BFC87900084C2200207C7900086E
:1058F00070B59AB005460846144601A900F0C2F8F2
:1059000001A8FCF7BDF9431C0022C6B25B0010469B
:10591000C5E9003423700323023404F8013C01ABD1
:10592000D1B202348E4201D81AB070BD13F8011BF7
:10593000013204F8010C04F8021CF1E708B5302329
:1059400083F311880348FFF713FA002383F31188C8
:1059500008BD00BF6055002090F8803003F01F02A2
:10596000012A07D190F881200B2A03D10023C0E936
:105970001D3315E003F06003202B08D1B0F884300C
:105980002BB990F88120212A03D81F2A04D8FFF7C9
:10599000D1B9222AEBD0FAE7034A4267072282678D
:1059A000C3670120704700BF4322002007B50529C7
:1059B00017D8DFE801F0191603191920302383F3F3
:1059C0001188104A01210190FFF77AFA019802210B
:1059D0000D4AFFF775FA0D48FFF796F9002383F398
:1059E000118803B05DF804FB302383F31188074866
:1059F000FFF760F9F2E7302383F311880348FFF7DC
:105A000077F9EBE71C790008407900086055002021
:105A100038B50C4D0C4C2A460C4904F10800FFF730
:105A200067FF05F1CA0204F110000949FFF760FFA2
:105A300005F5CA7204F118000649BDE83840FFF7C1
:105A400057BF00BF386E00204C220020FC780008B1
:105A5000067900081179000870B5044608460D461D
:105A6000FCF70EF9C6B22046013403780BB918468C
:105A700070BD32462946FCF7EFF80028F3D101202B
:105A8000F6E700002DE9F04705460C46FCF7F8F86C
:105A90002A49C6B22846FFF7DFFF08B10936F6B239
:105AA00027492846FFF7D8FF08B11036F6B2632E13
:105AB0000BD8DFF88880DFF88890224FDFF890A0BD
:105AC0002E7846B92670BDE8F08729462046BDE805
:105AD000F04701F051BE252E2CD107224146284621
:105AE000FCF7BAF860B9184B224603F1100153F8DD
:105AF000040B8B4242F8040BF9D107351034DFE771
:105B0000082249462846FCF7A7F898B9A21C0F4B73
:105B1000197802320909C95D02F8041C13F8011B47
:105B200001F00F015345C95D02F8031CF0D1183490
:105B30000835C5E7013504F8016BC1E7E8790008CD
:105B400011790008F07900089677000800E8F11F45
:105B50000CE8F11FBFF34F8F044B1A695107FCD1BA
:105B6000D3F810215207F8D1704700BF002000522F
:105B700008B50D4B1B78ABB9FFF7ECFF0B4BDA68A0
:105B8000D10704D50A4A5A6002F188325A60D3F824
:105B90000C21D20706D5064AC3F8042102F1883247
:105BA000C3F8042108BD00BF9670002000200052F9
:105BB0002301674508B5114B1B78F3B9104B1A69DF
:105BC000510703D5DA6842F04002DA60D3F81021B9
:105BD000520705D5D3F80C2142F04002C3F80C213E
:105BE000FFF7B8FF064BDA6842F00102DA60D3F83B
:105BF0000C2142F00102C3F80C2108BD9670002070
:105C0000002000520F289ABF00F580604004002059
:105C1000704700004FF400307047000010207047BC
:105C20000F2808B50BD8FFF7EDFF00F50033026829
:105C3000013204D104308342F9D1012008BD002093
:105C4000FCE700000F2838B505463FD8FFF782FF74
:105C50001F4CFFF78DFF4FF0FF3307286361C4F837
:105C600014311DD82361FFF775FF030243F02403AD
:105C7000E360E36843F08003E36023695A07FCD4E0
:105C80002846FFF767FFFFF7BDFF4FF4003100F034
:105C900057F92846FFF78EFFBDE83840FFF7C0BF31
:105CA000C4F81031FFF756FFA0F108031B0243F0C0
:105CB0002403C4F80C31D4F80C3143F08003C4F849
:105CC0000C31D4F810315B07FBD4D9E7002038BD84
:105CD000002000522DE9F84F05460C46104645EAD3
:105CE0000203DE0602D00020BDE8F88F20F01F007E
:105CF000DFF8BCB0DFF8BCA0FFF73AFF04EB000808
:105D0000444503D10120FFF755FFEDE72022294646
:105D1000204601F0FFFC10B920352034F0E72B4677
:105D200005F120021F68791CDDD104339A42F9D1B4
:105D300005F178431B481C4EB3F5801F1B4B38BF41
:105D4000184603F1F80332BFD946D1461E46FFF785
:105D500001FF0760A5EB040C336804F11C0143F05C
:105D600002033360231FD9F8007017F00507FAD13A
:105D700053F8042F8B424CF80320F4D1BFF34F8F1C
:105D8000FFF7E8FE4FF0FF3320222146036028464C
:105D9000336823F00203336001F0BCFC0028BBD061
:105DA0003846B0E7142100520C2000521420005253
:105DB000102000521021005210B5084C237828B151
:105DC0001BB9FFF7D5FE0123237010BD002BFCD0BB
:105DD0002070BDE81040FFF7EDBE00BF96700020B8
:105DE00038B5054D00240334696855F80C0B00F0F4
:105DF000B9F8122CF7D138BD047A0008084601F032
:105E000081BC000070B5104E82B0FFF78BFB0546D9
:105E100001F08AF8326803469042336037BF0B4A7C
:105E20000A495168146836BF0131D1E90041516017
:105E30000419284641F100010191FFF77DFB20463E
:105E4000019902B070BD00BF98700020A0700020C2
:105E500070B5124E82B0FFF765FB054601F064F89D
:105E6000326803469042336037BF0D4A0C4951688F
:105E7000146836BF0131D1E9004151600419284648
:105E800041F100010191FFF757FB4FF47A720023B3
:105E900020460199FAF72CFA02B070BD98700020E4
:105EA000A07000200244074BD2B210B5904200D13E
:105EB00010BD441C00B253F8200041F8040BE0B2BE
:105EC000F4E700BF504000580E4B30B51C6F24045F
:105ED00005D41C6F1C671C6F44F400441C670A4CFB
:105EE00002442368D2B243F480732360074B90428C
:105EF00000D130BD441C51F8045B00B243F820507F
:105F0000E0B2F4E7004402580048025850400058FC
:105F100007B5012201A90020FFF7C4FF019803B0D3
:105F20005DF804FB13B50446FFF7F2FFA04205D06D
:105F3000012201A900200194FFF7C6FF02B010BDA5
:105F40000144BFF34F8F064B884204D3BFF34F8FFA
:105F5000BFF36F8F7047C3F85C022030F4E700BFD7
:105F600000ED00E00144BFF34F8F064B884204D39D
:105F7000BFF34F8FBFF36F8F7047C3F870022030AD
:105F8000F4E700BF00ED00E070470000074B45F26A
:105F900055521A6002225A6040F6FF729A604CF61F
:105FA000CC421A600122024B1A7070470048005818
:105FB000AC700020034B1B781BB1034B4AF6AA229E
:105FC0001A607047AC70002000480058034B1A68F4
:105FD0001AB9034AD2F8D0241A607047A87000207A
:105FE00000400258024B4FF48032C3F8D02470476F
:105FF0000040025808B5FFF7E9FF024B1868C0F3EC
:10600000806008BDA870002070B5BFF34F8FBFF34C
:106010006F8F1A4A0021C2F85012BFF34F8FBFF39F
:106020006F8F536943F400335361BFF34F8FBFF356
:106030006F8FC2F88410BFF34F8FD2F8803043F6D1
:10604000E074C3F3C900C3F34E335B0103EA0406F3
:10605000014646EA81750139C2F86052F9D2203B07
:1060600013F1200FF2D1BFF34F8F536943F4803304
:106070005361BFF34F8FBFF36F8F70BD00ED00E032
:10608000FEE70000214B2248224A70B5904237D3E8
:10609000214BC11EDA1C121A22F003028B4238BFB8
:1060A00000220021FBF7F4FD1C4A0023C2F88430D3
:1060B000BFF34F8FD2F8803043F6E074C3F3C900CA
:1060C000C3F34E335B0103EA0406014646EA8175D9
:1060D0000139C2F86C52F9D2203B13F1200FF2D1F2
:1060E000BFF34F8FBFF36F8FBFF34F8FBFF36F8F30
:1060F0000023C2F85032BFF34F8FBFF36F8F70BDD4
:1061000053F8041B40F8041BC0E700BFA07C000844
:1061100080720020807200208072002000ED00E07C
:10612000054B996B21EA000199631A6E22EA00027D
:106130001A661B6E704700BF0045025870B5D0E963
:10614000244300224FF0FF359E6804EB42135101B7
:10615000D3F80009002805DAD3F8000940F08040A0
:10616000C3F80009D3F8000B002805DAD3F8000BB8
:1061700040F08040C3F8000B013263189642C3F828
:106180000859C3F8085BE0D24FF00113C4F81C387B
:1061900070BD0000890141F02001016103699B0687
:1061A000FCD41220FFF7D8B910B50A4C2046FEF7F0
:1061B00065FE094BC4F89030084BC4F89430084C85
:1061C0002046FEF75BFE074BC4F89030064BC4F840
:1061D000943010BDB070002000000840707A0008B4
:1061E0004C710020000004407C7A000870B50378F0
:1061F0000546012B58D13F4BD0F89040984254D1DE
:106200003D4B0E2165209A6B42F000629A631A6E34
:1062100042F000621A661B6E384BD3F8802042F0C1
:106220000062C3F88020D3F8802022F00062C3F817
:106230008020D3F88030FEF79DFA314BE360314B7C
:10624000C4F800380023D5F89060C4F8003EC0239D
:1062500023604FF40413A3633369002BFCDA01239A
:106260000C203361FFF778F93369DB07FCD4122087
:10627000FFF772F93369002BFCDA00262846A66086
:10628000FFF75CFF6B68C4F81068DB68C4F814683B
:10629000C4F81C6863BB1C4BA3614FF0FF33636100
:1062A000A36843F00103A36070BD184B9842C9D1A5
:1062B000114B4FF080609A6B42F000729A631A6E35
:1062C00042F000721A661B6E0C4BD3F8802042F02D
:1062D0000072C3F88020D3F8802022F00072C3F847
:1062E0008020D3F88030FFF71BFF0E214D20A2E75E
:1062F000074BD1E7B0700020004502580044025817
:106300004014004003002002003C30C04C710020CB
:10631000083C30C0F8B5D0F89040054600214FF059
:1063200000662046FFF736FFD5F8941000234FF0A3
:1063300001128F684FF0FF30C4F83438C4F81C28BD
:1063400004EB431201339F42C2F80069C2F8006BAC
:10635000C2F80809C2F8080BF2D20B68D5F89020F1
:10636000C5F89830636210231361166916F01006A1
:10637000FBD11220FFF7F0F8D4F8003823F4FE63C5
:10638000C4F80038A36943F4402343F01003A36129
:106390000923C4F81038C4F814380B4BEB604FF0E5
:1063A000C043C4F8103B094BC4F8003BC4F8106963
:1063B000C4F80039D5F8983003F1100243F4801383
:1063C000C5F89820A362F8BD4C7A00084080001000
:1063D000D0F8902090F88A10D2F8003823F4FE63A9
:1063E00043EA0113C2F80038704700002DE9F84372
:1063F00000EB8103D0F890500C468046DA680FFA23
:1064000081F94801166806F00306731E022B05EB9E
:1064100041134FF0000194BFB604384EC3F8101B6F
:106420004FF0010104F1100398BF06F1805601FA04
:1064300003F3916998BF06F5004600293AD0578AC0
:1064400004F15801374349016F50D5F81C180B432C
:106450000021C5F81C382B180127C3F81019A740D4
:106460005369611E9BB3138A928B9B08012A88BFD4
:106470005343D8F89820981842EA034301F14002A8
:106480002146C8F89800284605EB82025360FFF7C2
:1064900081FE08EB8900C3681B8A43EA84534834B1
:1064A0001E4364012E51D5F81C381F43C5F81C78D3
:1064B000BDE8F88305EB4917D7F8001B21F400412C
:1064C000C7F8001BD5F81C1821EA0303C0E704F144
:1064D0003F030B4A2846214605EB83035A60FFF72A
:1064E00059FE05EB4910D0F8003923F40043C0F8F9
:1064F0000039D5F81C3823EA0707D7E700800010D9
:1065000000040002D0F894201268C0F89820FFF729
:1065100015BE00005831D0F8903049015B5813F493
:10652000004004D013F4001F0CBF0220012070476C
:106530004831D0F8903049015B5813F4004004D042
:1065400013F4001F0CBF02200120704700EB8101F3
:10655000CB68196A0B6813604B6853607047000082
:1065600000EB810330B5DD68AA691368D36019B9FF
:10657000402B84BF402313606B8A1468D0F89020AE
:106580001C4402EB4110013C09B2B4FBF3F4634339
:10659000033323F0030343EAC44343F0C043C0F88A
:1065A000103B2B6803F00303012B0ED1D2F80838FF
:1065B00002EB411013F4807FD0F8003B14BF43F08E
:1065C000805343F00053C0F8003B02EB4112D2F875
:1065D000003B43F00443C2F8003B30BD2DE9F041DD
:1065E000D0F8906005460C4606EB4113D3F8087BC3
:1065F0003A07C3F8087B08D5D6F814381B0704D52A
:1066000000EB8103DB685B689847FA071FD5D6F873
:106610001438DB071BD505EB8403D968CCB98B692B
:10662000488A5A68B2FBF0F600FB16228AB918684D
:10663000DA6890420DD2121AC3E90024302383F3A2
:10664000118821462846FFF78BFF84F31188BDE8A7
:10665000F081012303FA04F26B8923EA02036B81C0
:10666000CB68002BF3D021462846BDE8F0411847FF
:1066700000EB81034A0170B5DD68D0F890306C6999
:106680002668E66056BB1A444FF40020C2F8100991
:106690002A6802F00302012A0AB20ED1D3F80808D0
:1066A00003EB421410F4807FD4F8000914BF40F0CB
:1066B000805040F00050C4F8000903EB4212D2F8B9
:1066C000000940F00440C2F800090122D3F8340860
:1066D00002FA01F10143C3F8341870BD19B9402E14
:1066E00084BF4020206020681A442E8A8419013C0F
:1066F000B4FBF6F440EAC44040F00050C6E70000A6
:106700002DE9F843D0F8906005460C464F0106EBA2
:106710004113D3F8088918F0010FC3F808891CD079
:10672000D6F81038DB0718D500EB8103D3F80CC07E
:10673000DCF81430D3F800E0DA68964530D2A2EBEA
:106740000E024FF000091A60C3F80490302383F35F
:106750001188FFF78DFF89F3118818F0800F1DD085
:10676000D6F834380126A640334217D005EB84030F
:106770000134D5F89050D3F80CC0E4B22F44DCF8C3
:10678000142005EB0434D2F800E05168714514D3AD
:10679000D5F8343823EA0606C5F83468BDE8F8832E
:1067A000012303FA01F2038923EA02030381DCF8DF
:1067B0000830002BD1D09847CFE7AEEB0103BCF8EF
:1067C0001000834228BF0346D7F8180980B2B3EB04
:1067D000800FE3D89068A0F1040959F8048FC4F839
:1067E0000080A0EB09089844B8F1040FF5D81844CC
:1067F0000B4490605360C8E72DE9F84FD0F89050F3
:1068000004466E69AB691E4016F480586E6103D071
:10681000BDE8F84FFEF7A2BB002E12DAD5F8003E15
:106820009B0705D0D5F8003E23F00303C5F8003ED2
:10683000D5F80438204623F00103C5F80438FEF7E4
:10684000BBFB370505D52046FFF778FC2046FEF751
:10685000A1FBB0040CD5D5F8083813F0060FEB688F
:1068600023F470530CBF43F4105343F4A053EB6074
:1068700031071BD56368DB681BB9AB6923F00803DC
:10688000AB612378052B0CD1D5F8003E9A0705D0D3
:10689000D5F8003E23F00303C5F8003E2046FEF77E
:1068A0008BFB6368DB680BB120469847F30200F16D
:1068B000BA80B70226D5D4F8909000274FF0010A8D
:1068C00009EB4712D2F8003B03F44023B3F5802FC5
:1068D00011D1D2F8003B002B0DDA62890AFA07F3D6
:1068E00022EA0303638104EB8703DB68DB6813B1EF
:1068F0003946204698470137D4F89430FFB29B6858
:106900009F42DDD9F00619D5D4F89000026AC2F38F
:106910000A1702F00F0302F4F012B2F5802F00F014
:10692000CA80B2F5402F09D104EB8303002200F5A1
:106930008050DB681B6A974240F0B0803003D5F886
:10694000185835D5E90303D500212046FFF746FE48
:10695000AA0303D501212046FFF740FE6B0303D5B0
:1069600002212046FFF73AFE2F0303D503212046DC
:10697000FFF734FEE80203D504212046FFF72EFE80
:10698000A90203D505212046FFF728FE6A0203D598
:1069900006212046FFF722FE2B0203D507212046C1
:1069A000FFF71CFEEF0103D508212046FFF716FE76
:1069B000700340F1A780E90703D500212046FFF7C7
:1069C0009FFEAA0703D501212046FFF799FE6B071A
:1069D00003D502212046FFF793FE2F0703D503219D
:1069E0002046FFF78DFEEE0603D504212046FFF773
:1069F00087FEA80603D505212046FFF781FE69061C
:106A000003D506212046FFF77BFE2A0603D5072182
:106A10002046FFF775FEEB0574D520460821BDE83A
:106A2000F84FFFF76DBED4F890904FF0000B4FF089
:106A3000010AD4F894305FFA8BF79B689F423FF6C7
:106A400038AF09EB4713D3F8002902F44022B2F51E
:106A5000802F20D1D3F80029002A1CDAD3F800298E
:106A600042F09042C3F80029D3F80029002AFBDB4A
:106A70003946D4F89000FFF78DFB22890AFA07F314
:106A800022EA0303238104EB8703DB689B6813B1CD
:106A90003946204698470BF1010BCAE7910701D10F
:106AA000D0F80080072A02F101029CBF03F8018B95
:106AB0004FEA18283FE704EB830300F58050DA68BB
:106AC000D2F818C0DCF80820DCE9001CA1EB0C0CA3
:106AD00000218F4208D1DB689B699A683A449A602A
:106AE0005A683A445A6029E711F0030F01D1D0F8EF
:106AF00000808C4501F1010184BF02F8018B4FEA4F
:106B00001828E6E7BDE8F88F08B50348FFF774FEDC
:106B1000BDE80840FDF7F8BCB070002008B5034898
:106B2000FFF76AFEBDE80840FDF7EEBC4C7100209F
:106B3000D0F8903003EB4111D1F8003B43F400133F
:106B4000C1F8003B70470000D0F8903003EB4111D2
:106B5000D1F8003943F40013C1F800397047000040
:106B6000D0F8903003EB4111D1F8003B23F400132F
:106B7000C1F8003B70470000D0F8903003EB4111A2
:106B8000D1F8003923F40013C1F800397047000030
:106B900030B50433039C0172002104FB0325C1605E
:106BA000C0E90653049B0363059BC0E90000C0E9EC
:106BB0000422C0E90842C0E90A11436330BD000065
:106BC0000022416AC260C0E90411C0E90A226FF0E4
:106BD0000101FEF731BD0000D0E90432934201D13A
:106BE000C2680AB9181D7047002070470369196010
:106BF0000021C2680132C260C269134482699342B3
:106C0000036124BF436A0361FEF70ABD38B5044639
:106C10000D46E3683BB162690020131D1268A36250
:106C20001344E36207E0237A33B929462046FEF78E
:106C3000E7FC0028EDDA38BD6FF00100FBE700004B
:106C4000C368C269013BC3604369134482699342CC
:106C5000436124BF436A436100238362036B03B132
:106C60001847704770B53023044683F31188866A4D
:106C70003EB9FFF7CBFF054618B186F311882846C9
:106C800070BDA36AE26A13F8015B9342A36202D368
:106C90002046FFF7D5FF002383F31188EFE70000BC
:106CA0002DE9F84F04460E46174698464FF0300936
:106CB00089F311880025AA46D4F828B0BBF1000F4B
:106CC00009D141462046FFF7A1FF20B18BF311887F
:106CD0002846BDE8F88FD4E90A12A7EB050B521A33
:106CE000934528BF9346BBF1400F1BD9334601F1B2
:106CF000400251F8040B914243F8040BF9D1A36A06
:106D0000403640354033A362D4E90A239A4202D385
:106D10002046FFF795FF8AF31188BD42D8D289F348
:106D20001188C9E730465A46FAF78CFFA36A5E44D9
:106D30005D445B44A362E7E710B5029C0433017233
:106D400003FB0421C460C0E906130023C0E90A3331
:106D5000039B0363049BC0E90000C0E90422C0E96F
:106D60000842436310BD0000026A6FF00101C26077
:106D7000426AC0E904220022C0E90A22FEF75CBC94
:106D8000D0E904239A4201D1C26822B9184650F8CA
:106D9000043B0B60704700231846FAE7C3680021E4
:106DA000C2690133C36043691344826993424361FA
:106DB00024BF436A4361FEF733BC000038B5044684
:106DC0000D46E3683BB1236900201A1DA262E26907
:106DD0001344E36207E0237A33B929462046FEF7DD
:106DE0000FFC0028EDDA38BD6FF00100FBE7000072
:106DF00003691960C268013AC260C26913448269BA
:106E00009342036124BF436A036100238362036BDF
:106E100003B118477047000070B530230D46044693
:106E2000114683F31188866A2EB9FFF7C7FF10B1A8
:106E300086F3118870BDA36A1D70A36AE26A0133EC
:106E40009342A36204D3E16920460439FFF7D0FFDF
:106E5000002080F31188EDE72DE9F84F04460D4638
:106E6000904699464FF0300A8AF311880026B346BF
:106E7000A76A4FB949462046FFF7A0FF20B187F324
:106E800011883046BDE8F88FD4E90A073A1AA8EB12
:106E90000607974228BF1746402F1BD905F140032C
:106EA00055F8042B9D4240F8042BF9D1A36A4036D3
:106EB0004033A362D4E90A239A4204D3E16920460D
:106EC0000439FFF795FF8BF311884645D9D28AF331
:106ED0001188CDE729463A46FAF7B4FEA36A3D4445
:106EE0003E443B44A362E5E7D0E904239A4217D12C
:106EF000C3689BB1836A8BB1043B9B1A0ED01360AD
:106F0000C368013BC360C3691A4483699A42026142
:106F100024BF436A0361002383620123184670473C
:106F20000023FBE700F01CB9014B586A704700BF13
:106F3000000C0040034B002258631A610222DA6001
:106F4000704700BF000C0040014B0022DA60704720
:106F5000000C0040014B5863704700BF000C00401C
:106F6000FEE7000070B51B4B0025044686B0586054
:106F70000E4685620163FDF79FFA04F11003A560D8
:106F8000E562C4E904334FF0FF33C4E90044C4E9C7
:106F90000635FFF7C9FF2B46024604F134012046AF
:106FA000C4E9082380230C4A2565FEF7DFFA012394
:106FB0000A4AE06000920375684672680192B268FE
:106FC000CDE90223064BCDE90435FEF7F7FA06B00A
:106FD00070BD00BF58550020887A00088D7A0008DF
:106FE000616F0008024AD36A1843D062704700BF3D
:106FF000F05200204B6843608B688360CB68C360AD
:107000000B6943614B6903628B6943620B680360E0
:107010007047000008B53A4B40F2FF713948D3F889
:1070200088200A43C3F88820D3F8882022F4FF621E
:1070300022F00702C3F88820D3F88830324B1A6C4C
:107040000A431A649A6E0A439A66304A9B6E114646
:10705000FFF7D0FF00F5806002F11C01FFF7CAFFC7
:1070600000F5806002F13801FFF7C4FF00F5806091
:1070700002F15401FFF7BEFF00F5806002F17001DC
:10708000FFF7B8FF00F5806002F18C01FFF7B2FF57
:1070900000F5806002F1A801FFF7ACFF00F5806009
:1070A00002F1C401FFF7A6FF00F5806002F1E001E4
:1070B000FFF7A0FF00F5806002F1FC01FFF79AFFE7
:1070C00002F58C7100F58060FFF794FF00F006F97F
:1070D0000F4BD3F8902242F00102C3F89022D3F86C
:1070E000942242F00102C3F894220522C3F89820AA
:1070F0004FF06052C3F89C20064AC3F8A02008BD98
:10710000004402580000025800450258947A0008D2
:1071100000ED00E01F00080308B500F0BDFAFEF71F
:10712000D9F90C4BDA6B42F04002DA635A6E22F066
:1071300040025A665B6E084B1A6842F008021A60F9
:107140001A6842F004021A60FEF740FFBDE80840EA
:10715000FEF75EBC00450258001802487047000068
:107160000E4B9A6C42F008029A641A6F42F00802C1
:107170001A670B4A1B6FD36B43F00803D363C72214
:10718000084B9A624FF0FF32DA6200229A615A632A
:10719000DA605A6001225A611A607047004502584D
:1071A0000010005C000C0040094A08B51169D36862
:1071B0000B40D9B29B076FEA0101116107D530235B
:1071C00083F31188FEF7ACF9002383F3118808BD1F
:1071D000000C0040044BDA6B0243DA635A6E104332
:1071E00058665B6E704700BF004502583A4B4FF03F
:1071F000FF31D3F8802062F00042C3F88020D3F83A
:10720000802002F00042C3F88020D3F88020D3F819
:107210008420C3F88410D3F884200022C3F884208B
:10722000D3F88400D86F40F0FF4040F4FF0040F4F2
:10723000DF4040F07F00D867D86F20F0FF4020F497
:10724000FF0020F4DF4020F07F00D867D86FD3F82C
:1072500088006FEA40506FEA5050C3F88800D3F8B6
:107260008800C0F30A00C3F88800D3F88800D3F878
:107270009000C3F89010D3F89000C3F89020D3F892
:107280009000D3F89400C3F89410D3F89400C3F896
:107290009420D3F89400D3F89800C3F89810D3F84A
:1072A0009800C3F89820D3F89800D3F88C00C3F85E
:1072B0008C10D3F88C00C3F88C20D3F88C00D3F852
:1072C0009C00C3F89C10D3F89C10C3F89C20D3F802
:1072D0009C3000F0B5B900BF0044025808B5012247
:1072E000504BC3F80821504B5A6D42F002025A65C8
:1072F000DA6F42F00202DA670422DB6F4B4BDA608E
:107300005A689104FCD54A4A1A6001229A60494A97
:10731000DA6000221A614FF440429A61434B9A6945
:107320009204FCD51A6842F480721A60424B1A6FBC
:1073300012F4407F04D04FF480321A6700221A679B
:107340001A6842F001021A603B4B1A685007FCD5DC
:1073500000221A611A6912F03802FBD1012119606A
:107360004FF0804159605A67344ADA62344A1A61F0
:107370001A6842F480321A602F4B1A689103FCD5C8
:107380001A6842F480521A601A689204FCD52D4A99
:107390002D499A6200225A63196301F57C01DA6370
:1073A00001F5E77199635A64284A1A64284ADA6237
:1073B0001A6842F0A8521A601F4B1A6802F028524D
:1073C000B2F1285FF9D148229A614FF48862DA61FC
:1073D00040221A621F4ADA641F4A1A651F4A5A6518
:1073E0001F4A9A6532231F4A1360136803F00F0384
:1073F000022BFAD1104A136943F003031361136996
:1074000003F03803182BFAD14FF00050FFF7E2FEDB
:107410004FF08040FFF7DEFE4FF00040BDE808402F
:10742000FFF7D8BE008000510045025800480258BE
:1074300000C000F004000001004402580000FF01F9
:10744000008890083220600063020901470E050899
:10745000DD0BBF0120000020000001100910E0003A
:1074600000010110002000524FF0B04208B5D2F8E0
:10747000883003F00103C2F8883023B1044A13684E
:107480000BB150689847BDE80840FDF73DB800BF14
:10749000007200204FF0B04208B5D2F8883003F0F7
:1074A0000203C2F8883023B1044A93680BB1D06854
:1074B0009847BDE80840FDF727B800BF00720020DC
:1074C0004FF0B04208B5D2F8883003F00403C2F898
:1074D000883023B1044A13690BB150699847BDE85D
:1074E0000840FDF711B800BF007200204FF0B04215
:1074F00008B5D2F8883003F00803C2F8883023B109
:10750000044A93690BB1D0699847BDE80840FCF77D
:10751000FBBF00BF007200204FF0B04208B5D2F8A8
:10752000883003F01003C2F8883023B1044A136A8C
:107530000BB1506A9847BDE80840FCF7E5BF00BFB3
:10754000007200204FF0B04310B5D3F8884004F427
:107550007872C3F88820A30604D5124A936A0BB147
:10756000D06A9847600604D50E4A136B0BB1506B76
:107570009847210604D50B4A936B0BB1D06B984703
:10758000E20504D5074A136C0BB1506C9847A3056C
:1075900004D5044A936C0BB1D06C9847BDE81040F9
:1075A000FCF7B2BF007200204FF0B04310B5D3F823
:1075B000884004F47C42C3F88820620504D5164A4A
:1075C000136D0BB1506D9847230504D5124A936D86
:1075D0000BB1D06D9847E00404D50F4A136E0BB180
:1075E000506E9847A10404D50B4A936E0BB1D06E30
:1075F0009847620404D5084A136F0BB1506F98473F
:10760000230404D5044A936F0BB1D06F9847BDE8AB
:107610001040FCF779BF00BF0072002008B5034896
:10762000FDF722F8BDE80840FCF76EBF804E002051
:1076300008B5FFF7B9FDBDE80840FCF765BF0000DD
:10764000062108B50846FDF795F806210720FDF745
:1076500091F806210820FDF78DF806210920FDF795
:1076600089F806210A20FDF785F806211720FDF785
:1076700081F806212820FDF77DF809217A20FDF701
:1076800079F807213220FDF775F80C215220BDE86A
:107690000840FDF76FB8000008B5FFF7A7FD00F040
:1076A0000DF8FDF70FFAFDF7E7FBFDF7B9FAFFF765
:1076B00055FDBDE80840FFF735BC00000023054A32
:1076C00019460133102BC2E9001102F10802F8D16A
:1076D000704700BF007200200B460146184600F0BC
:1076E00003B8000000F00EB810B5054C13462CB1DD
:1076F0000A4601460220AFF3008010BD2046FCE799
:1077000000000000024B01461868FEF777BB00BF7F
:107710006C22002010B501390244904201D10020B2
:1077200005E0037811F8014FA34201D0181B10BDEA
:107730000130F2E72DE9F041A3B1C91A17780144ED
:10774000044603F1FF3C8C42204601D9002009E0A9
:107750000578BD4204F10104F5D10CEB0405D618FF
:10776000A54201D1BDE8F08115F8018D16F801EDB3
:10777000F045F5D0E7E70000034611F8012B03F8C8
:10778000012B002AF9D170476F72672E6172647500
:1077900070696C6F742E4375626550696C6F742DDF
:1077A00043414E4D6F64000053544D333248373FD0
:1077B0003F3F0053544D3332483733782F373278B8
:1077C0000053544D3332483734332F3735332F3746
:1077D0003530000001105A000310590001205800F4
:1077E0000320560040A2E4F1646891060041A3E53D
:1077F000F26569920700000043414E4644496661C4
:1078000063653A204D6573736167652052414D2071
:107810004F766572666C6F772100000042616420CC
:1078200043414E496661636520696E6465782E0048
:1078300000000000000000009D2C000879250008D1
:107840009533000871250008E9250008F92900088A
:1078500061270008B1250008B52500088D2500081E
:1078600075250008B929000899250008CD340008BD
:10787000A52500088D2900080096000000000000E2
:1078800000000000000000000000000000000000F8
:1078900000000000854A0008714A0008AD4A00084F
:1078A000994A0008A54A0008914A00087D4A000844
:1078B000694A0008B94A0008000000009D4B000812
:1078C000894B0008C54B0008B14B0008BD4B0008B0
:1078D000A94B0008954B0008814B0008D14B0008CC
:1078E0000000000001000000000000006330000004
:1078F000EC78000848530020585500204172647508
:1079000050696C6F740025424F415244252D424C02
:10791000002553455249414C25000000020000005B
:1079200000000000BD4D00082D4E00084000400042
:10793000086E0020186E0020020000000000000009
:107940000300000000000000754E00080000000069
:1079500010000000286E0020000000000100000060
:1079600000000000B070002001010200AD590008C5
:10797000BD580008595900083D590008430000004F
:107980008479000809024300020100C032090400A2
:10799000000102020100052400100105240100017C
:1079A000042402020524060001070582030800FFE3
:1079B00009040100020A000000070501024000005E
:1079C000070581024000000012000000D079000885
:1079D0001201100102000040091241570002010289
:1079E000030100000403090425424F4152442500CD
:1079F00030313233343536373839414243444546E5
:107A00000000000000000020000002000200000052
:107A10000001003000000000080000000000002409
:107A200000000800040000000004000000FC00004A
:107A30000200000000000430008000000800000088
:107A400000000038000001000100000000000000FC
:107A5000D14F00088952000835530008400040000B
:107A6000E8710020E871002001000000F87100209A
:107A7000800000004001000008000000000100003C
:107A800000100000080000006D61696E0069646C00
:107A9000650000000000802A00000000AAAAAAAA2F
:107AA00000000024FFFF00000000000000A00A000A
:107AB0000000000000000000AAAAAAAA000000001E
:107AC000FFFF0000000000000000000000000000B8
:107AD00000000000AAAAAAAA00000000FFFF000000
:107AE00000000000000000000A000000000000008C
:107AF000AAAAAAAA00000000FFFF00009900000047
:107B0000000000000080020000000000AAAAAAAA4B
:107B100000400100FFFF00000000007007000000AF
:107B20000000000000000000AAAAAAAA00000000AD
:107B3000FFFF000000000000000000000500000042
:107B400000000000A5AAAAAA00000000FCFF000097
:107B50000000000000000000000000000000000025
:107B6000AAAAAAAA00000000FFFF0000000000006F
:107B7000000000000000000000000000AAAAAAAA5D
:107B800000000000FFFF00000000000000000000F7
:107B90000000000000000000AAAAAAAA000000003D
:107BA000FFFF0000000000000000000000000000D7
:107BB00000000000AAAAAAAA00000000FFFF00001F
:107BC00000000000000000005887FF7F0100000057
:107BD0003704000000000000000018000000000052
:107BE000FE2A0100D2040000FF00000060550020C2
:107BF000804E002000000000A877000883040000E9
:107C0000B377000850040000C17700080096000018
:107C100000000800960000000008000004000000BA
:107C2000E4790008000000000000000000000000EF
:107C30000000000000000000000000007022002092
:107C40000000000000000000000000000000000034
:107C50000000000000000000000000000000000024
:107C60000000000000000000000000000000000014
:107C70000000000000000000000000000000000004
:107C800000000000000000000000000000000000F4
:107C900000000000000000000000000000000000E4
:00000001FF
